 unpack200

 Timestamp is ffffffff (Sun Feb  7 06:28:15 2106)

 Preferred load address is 00400000

 Start         Length     Name                   Class
 0001:00000000 00011a9dH .text$mn                CODE
 0002:00000000 00000150H .idata$5                DATA
 0002:00000150 00000004H .00cfg                  DATA
 0002:00000154 00000004H .CRT$XCA                DATA
 0002:00000158 00000004H .CRT$XCAA               DATA
 0002:0000015c 00000004H .CRT$XCZ                DATA
 0002:00000160 00000004H .CRT$XIA                DATA
 0002:00000164 00000004H .CRT$XIAA               DATA
 0002:00000168 00000004H .CRT$XIAC               DATA
 0002:0000016c 00000004H .CRT$XIZ                DATA
 0002:00000170 00000004H .CRT$XPA                DATA
 0002:00000174 00000004H .CRT$XPZ                DATA
 0002:00000178 00000004H .CRT$XTA                DATA
 0002:0000017c 00000004H .CRT$XTZ                DATA
 0002:00000180 00000000H .gfids$y                DATA
 0002:00000180 00007630H .rdata                  DATA
 0002:000077b0 00000004H .rdata$sxdata           DATA
 0002:000077b4 000002c4H .rdata$zzzdbg           DATA
 0002:00007a78 00000004H .rtc$IAA                DATA
 0002:00007a7c 00000004H .rtc$IZZ                DATA
 0002:00007a80 00000004H .rtc$TAA                DATA
 0002:00007a84 00000004H .rtc$TZZ                DATA
 0002:00007a88 00000048H .xdata$x                DATA
 0002:00007ad0 00000048H .edata                  DATA
 0002:00007b18 00000104H .idata$2                DATA
 0002:00007c1c 00000014H .idata$3                DATA
 0002:00007c30 00000150H .idata$4                DATA
 0002:00007d80 000005feH .idata$6                DATA
 0003:00000000 00000b58H .data                   DATA
 0003:00000b58 00000784H .bss                    DATA
 0004:00000000 00000060H .rsrc$01                DATA
 0004:00000060 00000318H .rsrc$02                DATA

  Address         Publics by Value              Rva+Base       Lib:Object

 0000:00000000       ___guard_fids_table        00000000     <absolute>
 0000:00000000       ___hybrid_code_map_count   00000000     <absolute>
 0000:00000000       ___guard_longjmp_table     00000000     <absolute>
 0000:00000000       ___hybrid_code_map         00000000     <absolute>
 0000:00000000       ___guard_fids_count        00000000     <absolute>
 0000:00000000       ___guard_iat_count         00000000     <absolute>
 0000:00000000       ___dynamic_value_reloc_table 00000000     <absolute>
 0000:00000000       ___enclave_config          00000000     <absolute>
 0000:00000000       ___guard_longjmp_count     00000000     <absolute>
 0000:00000000       ___guard_iat_table         00000000     <absolute>
 0000:00000000       ___hybrid_auxiliary_iat    00000000     <absolute>
 0000:00000000       ___volatile_metadata       00000000     <absolute>
 0000:00000001       ___safe_se_handler_count   00000001     <absolute>
 0000:00000100       ___guard_flags             00000100     <absolute>
 0000:00000000       ___ImageBase               00400000     <linker-defined>
 0001:00000b22       _deflate                   00401b22 f   deflate.obj
 0001:000013a3       _deflateEnd                004023a3 f   deflate.obj
 0001:00001426       _deflateInit2_             00402426 f   deflate.obj
 0001:00001638       _deflateReset              00402638 f   deflate.obj
 0001:00001659       _deflateResetKeep          00402659 f   deflate.obj
 0001:00001fec       _inflate_fast              00402fec f   inffast.obj
 0001:000023f4       _inflate                   004033f4 f   inflate.obj
 0001:00003a30       _inflateEnd                00404a30 f   inflate.obj
 0001:00003a6c       _inflateInit2_             00404a6c f   inflate.obj
 0001:00003b12       _inflateReset              00404b12 f   inflate.obj
 0001:00003b3b       _inflateReset2             00404b3b f   inflate.obj
 0001:00003bb3       _inflateResetKeep          00404bb3 f   inflate.obj
 0001:00003d25       _inflate_table             00404d25 f   inftrees.obj
 0001:0000414c       __tr_align                 0040514c f   trees.obj
 0001:00004223       __tr_flush_bits            00405223 f   trees.obj
 0001:00004228       __tr_flush_block           00405228 f   trees.obj
 0001:00004432       __tr_init                  00405432 f   trees.obj
 0001:0000448f       __tr_stored_block          0040548f f   trees.obj
 0001:00005886       _adler32                   00406886 f   zadler32.obj
 0001:0000588b       _adler32_z                 0040688b f   zadler32.obj
 0001:00005ac8       _crc32                     00406ac8 f   zcrc32.obj
 0001:00005acd       _crc32_z                   00406acd f   zcrc32.obj
 0001:00005db6       _zcalloc                   00406db6 f   zutil.obj
 0001:00005dc8       _zcfree                    00406dc8 f   zutil.obj
 0001:00005dd4       ?getIndex@cpool@@QAEPAUcpindex@@C@Z 00406dd4 f i bands.obj
 0001:00005df1       ?getIntCount@band@@QAEHH@Z 00406df1 f   bands.obj
 0001:00005ebe       ?getIntTotal@band@@QAEHXZ  00406ebe f   bands.obj
 0001:00005f35       ?getLong@band@@QAE_JAAU1@_N@Z 00406f35 f   bands.obj
 0001:00005f6a       ?getRefCommon@band@@QAEPAUentry@@PAUcpindex@@_N@Z 00406f6a f   bands.obj
 0001:00005fdb       ?initIndexes@band@@SAXPAUunpacker@@@Z 00406fdb f   bands.obj
 0001:00006020       ?makeBands@band@@SAPAU1@PAUunpacker@@@Z 00407020 f   bands.obj
 0001:000060a4       ?readData@band@@QAEXH@Z    004070a4 f   bands.obj
 0001:00006254       ?setIndex@band@@QAEXPAUcpindex@@@Z 00407254 f   bands.obj
 0001:0000625e       ?setIndexByTag@band@@QAEXC@Z 0040725e f   bands.obj
 0001:0000627a       ?compareTo@bytes@@QAEHAAU1@@Z 0040727a f   bytes.obj
 0001:000062b1       ?copyFrom@bytes@@QAEXPBXII@Z 004072b1 f   bytes.obj
 0001:000062cb       ?ensureSize@fillbytes@@QAEXI@Z 004072cb f   bytes.obj
 0001:000062eb       ?free@bytes@@QAEXXZ        004072eb f   bytes.obj
 0001:0000630d       ?freeAll@ptrlist@@QAEXXZ   0040730d f   bytes.obj
 0001:0000634a       ?grow@fillbytes@@QAEPACI@Z 0040734a f   bytes.obj
 0001:000063e1       ?indexOf@ptrlist@@QAEHPBX@Z 004073e1 f   bytes.obj
 0001:00006407       ?malloc@bytes@@QAEXI@Z     00407407 f   bytes.obj
 0001:00006456       ?realloc@bytes@@QAEXI@Z    00407456 f   bytes.obj
 0001:000064ec       ?saveFrom@bytes@@QAEXPBXI@Z 004074ec f   bytes.obj
 0001:00006514       ?writeTo@bytes@@QAEPACPAC@Z 00407514 f   bytes.obj
 0001:0000655b       ?findByIndex@coding@@SAPAU1@H@Z 0040755b f   coding.obj
 0001:00006578       ?findBySpec@coding@@SAPAU1@H@Z 00407578 f   coding.obj
 0001:000065d3       ?findBySpec@coding@@SAPAU1@HHHH@Z 004075d3 f   coding.obj
 0001:00006618       ?free@coding@@QAEXXZ       00407618 f   coding.obj
 0001:0000664f       ?getInt@value_stream@@QAEHXZ 0040764f f   coding.obj
 0001:000068be       ?init@coding@@QAEPAU1@XZ   004078be f   coding.obj
 0001:00006b0b       ?init@coding_method@@QAEXAAPACPAC0HPAUcoding@@HPAUintlist@@@Z 00407b0b f   coding.obj
 0001:000071ae       ?init@value_stream@@QAEXPAC0PAUcoding@@@Z 004081ae f   coding.obj
 0001:000071d0       ?parse@coding@@SAIAAPACHH@Z 004081d0 f   coding.obj
 0001:00007234       ?parseMultiple@coding@@SAXAAPACHPACHH@Z 00408234 f   coding.obj
 0001:000072bf       ?parse_lgH@coding@@SAIAAPACHHH@Z 004082bf f   coding.obj
 0001:00007320       ?reset@coding_method@@QAEXPAUvalue_stream@@@Z 00408320 f   coding.obj
 0001:00007342       ?setCoding@value_stream@@QAEXPAUcoding@@@Z 00408342 f   coding.obj
 0001:00007442       ?sumInUnsignedRange@coding@@QAEHHH@Z 00408442 f   coding.obj
 0001:0000746e       ?current@unpacker@@SAPAU1@XZ 0040846e f   main.obj
 0001:000077c9       ?run@unpacker@@SAHHPAPAD@Z 004087c9 f   main.obj
 0001:00007cd4       ?saveIntStr@unpacker@@QAEPBDH@Z 00408cd4 f i main.obj
 0001:00007d15       ?saveStr@unpacker@@QAEPBDPBD@Z 00408d15 f i main.obj
 0001:00007d9a       ___local_stdio_printf_options 00408d9a f i main.obj
 0001:00007da0       __vfprintf_l               00408da0 f i main.obj
 0001:00007dc4       __vsnprintf_l              00408dc4 f i main.obj
 0001:00007df7       _fprintf                   00408df7 f i main.obj
 0001:00007e0f       _main                      00408e0f f   main.obj
 0001:00007e14       _sprintf                   00408e14 f i main.obj
 0001:00007e2e       ?abort@attr_definitions@unpacker@@QAEXPBD@Z 00408e2e f i unpack.obj
 0001:00007e3a       ?abort@cpool@@QAEXPBD@Z    00408e3a f i unpack.obj
 0001:00007e4a       ?abort@unpacker@@QAEXPBD@Z 00408e4a f   unpack.obj
 0001:00007e7c       ?add_size@@YAIIIH@Z        00408e7c f i unpack.obj
 0001:00007eb3       ?append@fillbytes@@QAEAAU1@PBXI@Z 00408eb3 f i unpack.obj
 0001:00007ed6       ?buildBands@attr_definitions@unpacker@@QAEPAPAUband@@PAUlayout_definition@2@@Z 00408ed6 f   unpack.obj
 0001:00007fee       ?calloc_heap@unpacker@@QAEPAXII_N0@Z 00408fee f   unpack.obj
 0001:000080a6       ?checkLegacy@unpacker@@QAEXPBD@Z 004090a6 f   unpack.obj
 0001:000080fa       ?check_options@unpacker@@QAEXXZ 004090fa f   unpack.obj
 0001:00008137       ?close_output@unpacker@@QAEPAUfillbytes@@PAU2@@Z 00409137 f   unpack.obj
 0001:0000821a       ?computeOutputIndexes@cpool@@QAEXXZ 0040921a f   unpack.obj
 0001:00008272       ?defineLayout@attr_definitions@unpacker@@QAEPAUlayout_definition@2@HPAUentry@@PBD@Z 00409272 f i unpack.obj
 0001:0000829e       ?defineLayout@attr_definitions@unpacker@@QAEPAUlayout_definition@2@HPBD0@Z 0040929e f   unpack.obj
 0001:00008388       ?dump_options@unpacker@@QAEXXZ 00409388 f   unpack.obj
 0001:000083d8       ?ensureClass@cpool@@QAEPAUentry@@AAUbytes@@@Z 004093d8 f   unpack.obj
 0001:00008464       ?ensureUtf8@cpool@@QAEPAUentry@@AAUbytes@@@Z 00409464 f   unpack.obj
 0001:000084d2       ?ensure_input@unpacker@@QAE_N_J@Z 004094d2 f   unpack.obj
 0001:0000862d       ?ensure_put_space@unpacker@@QAEXI@Z 0040962d f   unpack.obj
 0001:00008675       ?expandSignatures@cpool@@QAEXXZ 00409675 f   unpack.obj
 0001:00008824       ?finish@unpacker@@QAEXXZ   00409824 f   unpack.obj
 0001:00008902       ?free@attr_definitions@unpacker@@QAEXXZ 00409902 f i unpack.obj
 0001:00008975       ?free@jar@@QAEXXZ          00409975 f i unpack.obj
 0001:000089a0       ?free@unpacker@@QAEXXZ     004099a0 f   unpack.obj
 0001:00008b45       ?free_temps@unpacker@@QAEXXZ 00409b45 f i unpack.obj
 0001:00008b58       ?get@cpindex@@QAEPAUentry@@I@Z 00409b58 f   unpack.obj
 0001:00008b7d       ?getCount@attr_definitions@unpacker@@QAEAAHI@Z 00409b7d f i unpack.obj
 0001:00008b9d       ?getFieldIndex@cpool@@QAEPAUcpindex@@PAUentry@@@Z 00409b9d f i unpack.obj
 0001:00008bbf       ?getFirstChildIC@cpool@@QAEPAUinner_class@@PAUentry@@@Z 00409bbf f   unpack.obj
 0001:00008bdf       ?getIC@cpool@@QAEPAUinner_class@@PAUentry@@@Z 00409bdf f   unpack.obj
 0001:00008bff       ?getKQIndex@cpool@@QAEPAUcpindex@@XZ 00409bff f   unpack.obj
 0001:00008c75       ?getLayout@attr_definitions@unpacker@@QAEPAUlayout_definition@2@I@Z 00409c75 f i unpack.obj
 0001:00008c90       ?getMethodIndex@cpool@@QAEPAUcpindex@@PAUentry@@@Z 00409c90 f i unpack.obj
 0001:00008cbb       ?get_abort_message@unpacker@@QAEPBDXZ 00409cbb f   unpack.obj
 0001:00008cbf       ?get_code_header@unpacker@@QAEXAAH000@Z 00409cbf f   unpack.obj
 0001:00008d5c       ?get_next_file@unpacker@@QAEPAUfile@1@XZ 00409d5c f   unpack.obj
 0001:000090c2       ?get_option@unpacker@@QAEPBDPBD@Z 0040a0c2 f   unpack.obj
 0001:00009176       ?hashTabRef@cpool@@QAEAAPAUentry@@CAAUbytes@@@Z 0040a176 f   unpack.obj
 0001:00009232       ?init@band@@QAEXPAUunpacker@@HH@Z 0040a232 f i unpack.obj
 0001:0000925a       ?init@cpool@@QAEXPAUunpacker@@QAH@Z 0040a25a f   unpack.obj
 0001:000093d2       ?init@unpacker@@QAEXP6A_JPAU1@PAX_J2@Z@Z 0040a3d2 f   unpack.obj
 0001:00009448       ?initGroupIndexes@cpool@@QAEXXZ 0040a448 f   unpack.obj
 0001:0000950f       ?initMemberIndexes@cpool@@QAEXXZ 0040a50f f   unpack.obj
 0001:00009772       ?isIndex@attr_definitions@unpacker@@QAE_NI@Z 0040a772 f i unpack.obj
 0001:000097c4       ?isPredefined@attr_definitions@unpacker@@QAE_NI@Z 0040a7c4 f i unpack.obj
 0001:000097ef       ?isRedefined@attr_definitions@unpacker@@QAE_NI@Z 0040a7ef f i unpack.obj
 0001:00009884       ?parseIntLayout@attr_definitions@unpacker@@QAEPBDPBDAAPAUband@@C_N@Z 0040a884 f   unpack.obj
 0001:00009959       ?parseLayout@attr_definitions@unpacker@@QAEPBDPBDAAPAPAUband@@H@Z 0040a959 f   unpack.obj
 0001:0000a04f       ?parseNumeral@attr_definitions@unpacker@@QAEPBDPBDAAH@Z 0040b04f f   unpack.obj
 0001:0000a0e3       ?popBody@attr_definitions@unpacker@@QAEPAPAUband@@H@Z 0040b0e3 f   unpack.obj
 0001:0000a161       ?predefCount@attr_definitions@unpacker@@QAEHI@Z 0040b161 f   unpack.obj
 0001:0000a180       ?put_bytes@unpacker@@QAEXAAUbytes@@@Z 0040b180 f i unpack.obj
 0001:0000a199       ?put_label@unpacker@@QAEXHH@Z 0040b199 f   unpack.obj
 0001:0000a1e7       ?put_space@unpacker@@QAEPACI@Z 0040b1e7 f   unpack.obj
 0001:0000a21c       ?put_stackmap_type@unpacker@@QAEXXZ 0040b21c f   unpack.obj
 0001:0000a28f       ?putlayout@unpacker@@QAEXPAPAUband@@@Z 0040b28f f   unpack.obj
 0001:0000a49a       ?putref@unpacker@@QAEXPAUentry@@@Z 0040b49a f   unpack.obj
 0001:0000a4be       ?putref_index@unpacker@@QAEHPAUentry@@H@Z 0040b4be f   unpack.obj
 0001:0000a542       ?putu1ref@unpacker@@QAEXPAUentry@@@Z 0040b542 f   unpack.obj
 0001:0000a563       ?putu2@unpacker@@QAEXH@Z   0040b563 f   unpack.obj
 0001:0000a579       ?putu2_at@unpacker@@SAXPACH@Z 0040b579 f   unpack.obj
 0001:0000a5a2       ?putu4@unpacker@@QAEXH@Z   0040b5a2 f   unpack.obj
 0001:0000a5b8       ?putu4_at@unpacker@@SAXPACH@Z 0040b5b8 f   unpack.obj
 0001:0000a5db       ?putu8@unpacker@@QAEX_J@Z  0040b5db f   unpack.obj
 0001:0000a5f6       ?putu8_at@unpacker@@SAXPAC_J@Z 0040b5f6 f   unpack.obj
 0001:0000a617       ?readBandData@attr_definitions@unpacker@@QAEXH@Z 0040b617 f   unpack.obj
 0001:0000a6aa       ?readBandData@attr_definitions@unpacker@@QAEXPAPAUband@@I@Z 0040b6aa f   unpack.obj
 0001:0000a7e3       ?read_Utf8_values@unpacker@@QAEXPAUentry@@HC@Z 0040b7e3 f i unpack.obj
 0001:0000ada7       ?read_attr_defs@unpacker@@QAEXXZ 0040bda7 f   unpack.obj
 0001:0000b05e       ?read_attrs@unpacker@@QAEXHH@Z 0040c05e f   unpack.obj
 0001:0000b9fb       ?read_bands@unpacker@@QAEXXZ 0040c9fb f   unpack.obj
 0001:0000ba67       ?read_bcs@unpacker@@QAEXXZ 0040ca67 f i unpack.obj
 0001:0000bda3       ?read_bootstrap_methods@unpacker@@QAEXPAUentry@@HC@Z 0040cda3 f   unpack.obj
 0001:0000bee0       ?read_classes@unpacker@@QAEXXZ 0040cee0 f   unpack.obj
 0001:0000c00e       ?read_code_headers@unpacker@@QAEXXZ 0040d00e f   unpack.obj
 0001:0000c177       ?read_cp@unpacker@@QAEXXZ  0040d177 f   unpack.obj
 0001:0000c44b       ?read_double_refs@unpacker@@QAEXAAUband@@CCPAUentry@@HC@Z 0040d44b f   unpack.obj
 0001:0000c515       ?read_double_words@unpacker@@QAEXAAUband@@PAUentry@@HCH@Z 0040d515 f   unpack.obj
 0001:0000c5a6       ?read_file_header@unpacker@@QAEXXZ 0040d5a6 f   unpack.obj
 0001:0000cd98       ?read_files@unpacker@@QAEXXZ 0040dd98 f   unpack.obj
 0001:0000ce93       ?read_ics@unpacker@@QAEXXZ 0040de93 f   unpack.obj
 0001:0000d1fb       ?read_method_handle@unpacker@@QAEXPAUentry@@HCH@Z 0040e1fb f   unpack.obj
 0001:0000d2f0       ?read_method_type@unpacker@@QAEXPAUentry@@HCH@Z 0040e2f0 f   unpack.obj
 0001:0000d3bb       ?read_signature_values@unpacker@@QAEXPAUentry@@HC@Z 0040e3bb f   unpack.obj
 0001:0000d53c       ?read_single_refs@unpacker@@QAEXAAUband@@CPAUentry@@HCH@Z 0040e53c f   unpack.obj
 0001:0000d640       ?read_single_words@unpacker@@QAEXAAUband@@PAUentry@@HCH@Z 0040e640 f i unpack.obj
 0001:0000d6ba       ?redirect_stdio@unpacker@@QAEXXZ 0040e6ba f   unpack.obj
 0001:0000d752       ?ref_band_for_op@unpacker@@QAEPAUband@@H@Z 0040e752 f   unpack.obj
 0001:0000d88e       ?ref_band_for_self_op@unpacker@@QAEPAUband@@HAA_NAAH@Z 0040e88e f   unpack.obj
 0001:0000d905       ?requestOutputIndex@entry@@QAEXAAUcpool@@H@Z 0040e905 f   unpack.obj
 0001:0000d976       ?reset@unpacker@@QAEXXZ    0040e976 f   unpack.obj
 0001:0000dbae       ?resetOutputIndexes@cpool@@QAEXXZ 0040ebae f   unpack.obj
 0001:0000dc03       ?reset_cur_classfile@unpacker@@QAEXXZ 0040ec03 f   unpack.obj
 0001:0000dc4b       ?saveTo@unpacker@@QAEXAAUbytes@@PACI@Z 0040ec4b f   unpack.obj
 0001:0000dc9d       ?scale_size@@YAIII@Z       0040ec9d f i unpack.obj
 0001:0000dcbe       ?set_option@unpacker@@QAE_NPBD0@Z 0040ecbe f   unpack.obj
 0001:0000de0d       ?set_output@unpacker@@QAEXPAUfillbytes@@@Z 0040ee0d f i unpack.obj
 0001:0000de44       ?start@unpacker@@QAEXPAXI@Z 0040ee44 f   unpack.obj
 0001:0000decd       ?to_bci@unpacker@@QAEII@Z  0040eecd f   unpack.obj
 0001:0000df1b       ?typeSize@entry@@QAEHXZ    0040ef1b f   unpack.obj
 0001:0000df91       ?utf8String@entry@@QAEPBDXZ 0040ef91 f i unpack.obj
 0001:0000dfb5       ?write_attrs@unpacker@@QAEHH_K@Z 0040efb5 f   unpack.obj
 0001:0000ea27       ?write_bc_ops@unpacker@@QAEXXZ 0040fa27 f i unpack.obj
 0001:0000f1f6       ?write_bsms@unpacker@@QAEHHH@Z 004101f6 f   unpack.obj
 0001:0000f300       ?write_classfile_head@unpacker@@QAEXXZ 00410300 f   unpack.obj
 0001:0000f45a       ?write_classfile_tail@unpacker@@QAEXXZ 0041045a f   unpack.obj
 0001:0000f68f       ?write_code@unpacker@@QAEXXZ 0041068f f i unpack.obj
 0001:0000f866       ?write_file_to_jar@unpacker@@QAEXPAUfile@1@@Z 00410866 f   unpack.obj
 0001:0000fa08       ?write_ics@unpacker@@QAEHHH@Z 00410a08 f   unpack.obj
 0001:0000fd5f       ?write_members@unpacker@@QAEXHH@Z 00410d5f f   unpack.obj
 0001:0000fe99       __snprintf                 00410e99 f i unpack.obj
 0001:0000feb3       __vsnprintf                00410eb3 f i unpack.obj
 0001:0000fece       _outputEntry_cmp           00410ece f   unpack.obj
 0001:0000ff3f       _raw_address_cmp           00410f3f f   unpack.obj
 0001:0000ff5a       ?must_calloc@@YAPAXII@Z    00410f5a f   utils.obj
 0001:0000ff9d       ?unpack_abort@@YAXPBDPAUunpacker@@@Z 00410f9d f   utils.obj
 0001:0000ffe6       ?unpack_aborting@@YA_NPAUunpacker@@@Z 00410fe6 f   utils.obj
 0001:0001001b       ?addJarEntry@jar@@QAEXPBD_NHAAUbytes@@2@Z 0041101b f   zip.obj
 0001:0001011e       ?add_to_jar_directory@jar@@QAEXPBD_NHHHK@Z 0041111e f   zip.obj
 0001:00010269       ?closeJarFile@jar@@QAEX_N@Z 00411269 f   zip.obj
 0001:000102af       ?deflate_bytes@jar@@QAE_NAAUbytes@@0@Z 004112af f   zip.obj
 0001:000103af       ?dostime@jar@@QAEKHHHHHH@Z 004113af f i zip.obj
 0001:00010400       ?free@gunzip@@QAEXXZ       00411400 f   zip.obj
 0001:00010435       ?get_dostime@jar@@QAEKH@Z  00411435 f   zip.obj
 0001:000104dc       ?init@gunzip@@QAEXPAUunpacker@@@Z 004114dc f   zip.obj
 0001:00010540       ?init@jar@@QAEXPAUunpacker@@@Z 00411540 f   zip.obj
 0001:0001055e       ?openJarFile@jar@@QAEXPBD@Z 0041155e f   zip.obj
 0001:000105a3       ?read_fixed_field@gunzip@@QAEXPADI@Z 004115a3 f   zip.obj
 0001:0001082d       ?start@gunzip@@QAEXH@Z     0041182d f   zip.obj
 0001:0001091d       ?write_central_directory@jar@@QAEXXZ 0041191d f   zip.obj
 0001:00010aa5       ?write_data@jar@@QAEXPAXI@Z 00411aa5 f   zip.obj
 0001:00010afc       ?write_jar_extra@jar@@QAEXHHI@Z 00411afc f   zip.obj
 0001:00010b56       ?write_jar_header@jar@@QAEXPBD_NHHHI@Z 00411b56 f   zip.obj
 0001:00010c94       ___raise_securityfailure   00411c94 f   MSVCRT:gs_report.obj
 0001:00010cbc       ___report_gsfailure        00411cbc f   MSVCRT:gs_report.obj
 0001:00010db5       ___report_rangecheckfailure 00411db5 f   MSVCRT:gs_report.obj
 0001:00010dc1       ___report_securityfailure  00411dc1 f   MSVCRT:gs_report.obj
 0001:00010e8f       @__security_check_cookie@4 00411e8f f   MSVCRT:secchk.obj
 0001:00010ea0       __allrem                   00411ea0 f   MSVCRT:llrem.obj
 0001:00010f60       __allmul                   00411f60 f   MSVCRT:llmul.obj
 0001:00010fa0       __aullshr                  00411fa0 f   MSVCRT:ullshr.obj
 0001:00011206       _mainCRTStartup            00412206 f   MSVCRT:exe_main.obj
 0001:00011254       ___scrt_acquire_startup_lock 00412254 f   MSVCRT:utility.obj
 0001:00011286       ___scrt_initialize_crt     00412286 f   MSVCRT:utility.obj
 0001:000112bf       ___scrt_initialize_onexit_tables 004122bf f   MSVCRT:utility.obj
 0001:00011364       ___scrt_is_nonwritable_in_current_image 00412364 f   MSVCRT:utility.obj
 0001:000113f8       ___scrt_release_startup_lock 004123f8 f   MSVCRT:utility.obj
 0001:00011415       ___scrt_uninitialize_crt   00412415 f   MSVCRT:utility.obj
 0001:0001143d       __onexit                   0041243d f   MSVCRT:utility.obj
 0001:00011478       _atexit                    00412478 f   MSVCRT:utility.obj
 0001:000114da       ___security_init_cookie    004124da f   MSVCRT:gs_support.obj
 0001:00011525       ___scrt_stub_for_initialize_mta 00412525 f   MSVCRT:utility_desktop.obj
 0001:00011525       __get_startup_commit_mode  00412525 f   MSVCRT:commit_mode.obj
 0001:00011525       ___scrt_initialize_winrt   00412525 f   MSVCRT:utility_desktop.obj
 0001:00011525       ___scrt_exe_initialize_mta 00412525 f   MSVCRT:utility_desktop.obj
 0001:00011525       __get_startup_thread_locale_mode 00412525 f   MSVCRT:thread_locale.obj
 0001:00011525       __matherr                  00412525 f   MSVCRT:matherr.obj
 0001:00011525       __get_startup_new_mode     00412525 f   MSVCRT:new_mode.obj
 0001:00011528       __get_startup_argv_mode    00412528 f   MSVCRT:argv_mode.obj
 0001:0001152c       __get_startup_file_mode    0041252c f   MSVCRT:file_mode.obj
 0001:00011532       ?__scrt_initialize_type_info@@YAXXZ 00412532 f   MSVCRT:tncleanup.obj
 0001:0001153e       ___acrt_uninitialize       0041253e f   MSVCRT:ucrt_stubs.obj
 0001:0001153e       __should_initialize_environment 0041253e f   MSVCRT:env_mode.obj
 0001:0001153e       ___scrt_stub_for_acrt_uninitialize 0041253e f   MSVCRT:ucrt_stubs.obj
 0001:0001153e       ___vcrt_uninitialize       0041253e f   MSVCRT:ucrt_stubs.obj
 0001:0001153e       ___scrt_stub_for_acrt_initialize 0041253e f   MSVCRT:ucrt_stubs.obj
 0001:0001153e       ___vcrt_initialize         0041253e f   MSVCRT:ucrt_stubs.obj
 0001:0001153e       ___acrt_initialize         0041253e f   MSVCRT:ucrt_stubs.obj
 0001:00011541       __initialize_default_precision 00412541 f   MSVCRT:default_precision.obj
 0001:00011562       __initialize_denormal_control 00412562 f   MSVCRT:denormal_control.obj
 0001:00011562       __initialize_invalid_parameter_handler 00412562 f   MSVCRT:invalid_parameter_handler.obj
 0001:00011562       @_guard_check_icall_nop@4  00412562 f   MSVCRT:guard_support.obj
 0001:00011563       ___local_stdio_scanf_options 00412563 f i MSVCRT:default_local_stdio_options.obj
 0001:00011569       ___scrt_initialize_default_local_stdio_options 00412569 f   MSVCRT:default_local_stdio_options.obj
 0001:00011586       ___scrt_is_user_matherr_present 00412586 f   MSVCRT:matherr_detection.obj
 0001:00011592       ___scrt_get_dyn_tls_init_callback 00412592 f   MSVCRT:dyn_tls_init.obj
 0001:00011598       ___scrt_get_dyn_tls_dtor_callback 00412598 f   MSVCRT:dyn_tls_dtor.obj
 0001:0001159e       ___scrt_fastfail           0041259e f   MSVCRT:utility_desktop.obj
 0001:000116b8       ___scrt_initialize_mta     004126b8 f   MSVCRT:utility_desktop.obj
 0001:000116bd       ___scrt_is_managed_app     004126bd f   MSVCRT:utility_desktop.obj
 0001:00011700       ___scrt_set_unhandled_exception_filter 00412700 f   MSVCRT:utility_desktop.obj
 0001:0001170c       ___scrt_unhandled_exception_filter@4 0041270c f   MSVCRT:utility_desktop.obj
 0001:0001174d       __crt_debugger_hook        0041274d f   MSVCRT:utility_desktop.obj
 0001:00011755       __RTC_Initialize           00412755 f   MSVCRT:initsect.obj
 0001:00011781       __RTC_Terminate            00412781 f   MSVCRT:initsect.obj
 0001:000117b0       __SEH_prolog4              004127b0 f   MSVCRT:sehprolg4.obj
 0001:000117f6       __SEH_epilog4              004127f6 f   MSVCRT:sehprolg4.obj
 0001:0001180b       __except_handler4          0041280b f   MSVCRT:chandler4gs.obj
 0001:0001182e       ___isa_available_init      0041282e f   MSVCRT:cpu_disp.obj
 0001:000119c5       ___scrt_is_ucrt_dll_in_use 004129c5 f   MSVCRT:ucrt_detection.obj
 0001:000119d1       _IsProcessorFeaturePresent@4 004129d1 f   kernel32:KERNEL32.dll
 0001:000119d7       _memcpy                    004129d7 f   vcruntime:VCRUNTIME140.dll
 0001:000119dd       _memset                    004129dd f   vcruntime:VCRUNTIME140.dll
 0001:000119e3       _memcmp                    004129e3 f   vcruntime:VCRUNTIME140.dll
 0001:000119e9       _strchr                    004129e9 f   vcruntime:VCRUNTIME140.dll
 0001:000119ef       _strrchr                   004129ef f   vcruntime:VCRUNTIME140.dll
 0001:000119f5       __except_handler4_common   004129f5 f   vcruntime:VCRUNTIME140.dll
 0001:000119fb       _strcmp                    004129fb f   ucrt:api-ms-win-crt-string-l1-1-0.dll
 0001:00011a01       _strlen                    00412a01 f   ucrt:api-ms-win-crt-string-l1-1-0.dll
 0001:00011a07       _exit                      00412a07 f   ucrt:api-ms-win-crt-runtime-l1-1-0.dll
 0001:00011a0d       _strcat                    00412a0d f   ucrt:api-ms-win-crt-string-l1-1-0.dll
 0001:00011a13       __seh_filter_exe           00412a13 f   ucrt:api-ms-win-crt-runtime-l1-1-0.dll
 0001:00011a19       __set_app_type             00412a19 f   ucrt:api-ms-win-crt-runtime-l1-1-0.dll
 0001:00011a1f       ___setusermatherr          00412a1f f   ucrt:api-ms-win-crt-math-l1-1-0.dll
 0001:00011a25       __configure_narrow_argv    00412a25 f   ucrt:api-ms-win-crt-runtime-l1-1-0.dll
 0001:00011a2b       __initialize_narrow_environment 00412a2b f   ucrt:api-ms-win-crt-runtime-l1-1-0.dll
 0001:00011a31       __get_initial_narrow_environment 00412a31 f   ucrt:api-ms-win-crt-runtime-l1-1-0.dll
 0001:00011a37       __initterm                 00412a37 f   ucrt:api-ms-win-crt-runtime-l1-1-0.dll
 0001:00011a3d       __initterm_e               00412a3d f   ucrt:api-ms-win-crt-runtime-l1-1-0.dll
 0001:00011a43       __exit                     00412a43 f   ucrt:api-ms-win-crt-runtime-l1-1-0.dll
 0001:00011a49       __set_fmode                00412a49 f   ucrt:api-ms-win-crt-stdio-l1-1-0.dll
 0001:00011a4f       ___p___argc                00412a4f f   ucrt:api-ms-win-crt-runtime-l1-1-0.dll
 0001:00011a55       ___p___argv                00412a55 f   ucrt:api-ms-win-crt-runtime-l1-1-0.dll
 0001:00011a5b       __cexit                    00412a5b f   ucrt:api-ms-win-crt-runtime-l1-1-0.dll
 0001:00011a61       __c_exit                   00412a61 f   ucrt:api-ms-win-crt-runtime-l1-1-0.dll
 0001:00011a67       __register_thread_local_exe_atexit_callback 00412a67 f   ucrt:api-ms-win-crt-runtime-l1-1-0.dll
 0001:00011a6d       __configthreadlocale       00412a6d f   ucrt:api-ms-win-crt-locale-l1-1-0.dll
 0001:00011a73       __set_new_mode             00412a73 f   ucrt:api-ms-win-crt-heap-l1-1-0.dll
 0001:00011a79       ___p__commode              00412a79 f   ucrt:api-ms-win-crt-stdio-l1-1-0.dll
 0001:00011a7f       __initialize_onexit_table  00412a7f f   ucrt:api-ms-win-crt-runtime-l1-1-0.dll
 0001:00011a85       __register_onexit_function 00412a85 f   ucrt:api-ms-win-crt-runtime-l1-1-0.dll
 0001:00011a8b       __crt_atexit               00412a8b f   ucrt:api-ms-win-crt-runtime-l1-1-0.dll
 0001:00011a91       __controlfp_s              00412a91 f   ucrt:api-ms-win-crt-runtime-l1-1-0.dll
 0001:00011a97       _terminate                 00412a97 f   ucrt:api-ms-win-crt-runtime-l1-1-0.dll
 0002:00000000       __imp__UnhandledExceptionFilter@4 00413000     kernel32:KERNEL32.dll
 0002:00000004       __imp__SetUnhandledExceptionFilter@4 00413004     kernel32:KERNEL32.dll
 0002:00000008       __imp__GetCurrentProcess@0 00413008     kernel32:KERNEL32.dll
 0002:0000000c       __imp__TerminateProcess@8  0041300c     kernel32:KERNEL32.dll
 0002:00000010       __imp__IsProcessorFeaturePresent@4 00413010     kernel32:KERNEL32.dll
 0002:00000014       __imp__QueryPerformanceCounter@4 00413014     kernel32:KERNEL32.dll
 0002:00000018       __imp__GetCurrentProcessId@0 00413018     kernel32:KERNEL32.dll
 0002:0000001c       __imp__GetCurrentThreadId@0 0041301c     kernel32:KERNEL32.dll
 0002:00000020       __imp__GetSystemTimeAsFileTime@4 00413020     kernel32:KERNEL32.dll
 0002:00000024       __imp__InitializeSListHead@4 00413024     kernel32:KERNEL32.dll
 0002:00000028       __imp__IsDebuggerPresent@0 00413028     kernel32:KERNEL32.dll
 0002:0000002c       __imp__GetModuleHandleW@4  0041302c     kernel32:KERNEL32.dll
 0002:00000030       \177KERNEL32_NULL_THUNK_DATA 00413030     kernel32:KERNEL32.dll
 0002:00000034       __imp__memcpy              00413034     vcruntime:VCRUNTIME140.dll
 0002:00000038       __imp__memset              00413038     vcruntime:VCRUNTIME140.dll
 0002:0000003c       __imp__memcmp              0041303c     vcruntime:VCRUNTIME140.dll
 0002:00000040       __imp__strchr              00413040     vcruntime:VCRUNTIME140.dll
 0002:00000044       __imp__strrchr             00413044     vcruntime:VCRUNTIME140.dll
 0002:00000048       __imp___except_handler4_common 00413048     vcruntime:VCRUNTIME140.dll
 0002:0000004c       \177VCRUNTIME140_NULL_THUNK_DATA 0041304c     vcruntime:VCRUNTIME140.dll
 0002:00000050       __imp__atoi                00413050     ucrt:api-ms-win-crt-convert-l1-1-0.dll
 0002:00000054       \177api-ms-win-crt-convert-l1-1-0_NULL_THUNK_DATA 00413054     ucrt:api-ms-win-crt-convert-l1-1-0.dll
 0002:00000058       __imp__getenv              00413058     ucrt:api-ms-win-crt-environment-l1-1-0.dll
 0002:0000005c       \177api-ms-win-crt-environment-l1-1-0_NULL_THUNK_DATA 0041305c     ucrt:api-ms-win-crt-environment-l1-1-0.dll
 0002:00000060       __imp__remove              00413060     ucrt:api-ms-win-crt-filesystem-l1-1-0.dll
 0002:00000064       \177api-ms-win-crt-filesystem-l1-1-0_NULL_THUNK_DATA 00413064     ucrt:api-ms-win-crt-filesystem-l1-1-0.dll
 0002:00000068       __imp___set_new_mode       00413068     ucrt:api-ms-win-crt-heap-l1-1-0.dll
 0002:0000006c       __imp__calloc              0041306c     ucrt:api-ms-win-crt-heap-l1-1-0.dll
 0002:00000070       __imp__free                00413070     ucrt:api-ms-win-crt-heap-l1-1-0.dll
 0002:00000074       __imp__realloc             00413074     ucrt:api-ms-win-crt-heap-l1-1-0.dll
 0002:00000078       __imp__malloc              00413078     ucrt:api-ms-win-crt-heap-l1-1-0.dll
 0002:0000007c       \177api-ms-win-crt-heap-l1-1-0_NULL_THUNK_DATA 0041307c     ucrt:api-ms-win-crt-heap-l1-1-0.dll
 0002:00000080       __imp___configthreadlocale 00413080     ucrt:api-ms-win-crt-locale-l1-1-0.dll
 0002:00000084       \177api-ms-win-crt-locale-l1-1-0_NULL_THUNK_DATA 00413084     ucrt:api-ms-win-crt-locale-l1-1-0.dll
 0002:00000088       __imp____setusermatherr    00413088     ucrt:api-ms-win-crt-math-l1-1-0.dll
 0002:0000008c       \177api-ms-win-crt-math-l1-1-0_NULL_THUNK_DATA 0041308c     ucrt:api-ms-win-crt-math-l1-1-0.dll
 0002:00000090       __imp___controlfp_s        00413090     ucrt:api-ms-win-crt-runtime-l1-1-0.dll
 0002:00000094       __imp___crt_atexit         00413094     ucrt:api-ms-win-crt-runtime-l1-1-0.dll
 0002:00000098       __imp___errno              00413098     ucrt:api-ms-win-crt-runtime-l1-1-0.dll
 0002:0000009c       __imp__exit                0041309c     ucrt:api-ms-win-crt-runtime-l1-1-0.dll
 0002:000000a0       __imp___initialize_onexit_table 004130a0     ucrt:api-ms-win-crt-runtime-l1-1-0.dll
 0002:000000a4       __imp__abort               004130a4     ucrt:api-ms-win-crt-runtime-l1-1-0.dll
 0002:000000a8       __imp__terminate           004130a8     ucrt:api-ms-win-crt-runtime-l1-1-0.dll
 0002:000000ac       __imp___register_thread_local_exe_atexit_callback 004130ac     ucrt:api-ms-win-crt-runtime-l1-1-0.dll
 0002:000000b0       __imp___c_exit             004130b0     ucrt:api-ms-win-crt-runtime-l1-1-0.dll
 0002:000000b4       __imp___seh_filter_exe     004130b4     ucrt:api-ms-win-crt-runtime-l1-1-0.dll
 0002:000000b8       __imp___set_app_type       004130b8     ucrt:api-ms-win-crt-runtime-l1-1-0.dll
 0002:000000bc       __imp___register_onexit_function 004130bc     ucrt:api-ms-win-crt-runtime-l1-1-0.dll
 0002:000000c0       __imp___configure_narrow_argv 004130c0     ucrt:api-ms-win-crt-runtime-l1-1-0.dll
 0002:000000c4       __imp___initialize_narrow_environment 004130c4     ucrt:api-ms-win-crt-runtime-l1-1-0.dll
 0002:000000c8       __imp___get_initial_narrow_environment 004130c8     ucrt:api-ms-win-crt-runtime-l1-1-0.dll
 0002:000000cc       __imp___initterm           004130cc     ucrt:api-ms-win-crt-runtime-l1-1-0.dll
 0002:000000d0       __imp___initterm_e         004130d0     ucrt:api-ms-win-crt-runtime-l1-1-0.dll
 0002:000000d4       __imp___exit               004130d4     ucrt:api-ms-win-crt-runtime-l1-1-0.dll
 0002:000000d8       __imp___cexit              004130d8     ucrt:api-ms-win-crt-runtime-l1-1-0.dll
 0002:000000dc       __imp____p___argc          004130dc     ucrt:api-ms-win-crt-runtime-l1-1-0.dll
 0002:000000e0       __imp____p___argv          004130e0     ucrt:api-ms-win-crt-runtime-l1-1-0.dll
 0002:000000e4       \177api-ms-win-crt-runtime-l1-1-0_NULL_THUNK_DATA 004130e4     ucrt:api-ms-win-crt-runtime-l1-1-0.dll
 0002:000000e8       __imp____acrt_iob_func     004130e8     ucrt:api-ms-win-crt-stdio-l1-1-0.dll
 0002:000000ec       __imp__fwrite              004130ec     ucrt:api-ms-win-crt-stdio-l1-1-0.dll
 0002:000000f0       __imp__fseek               004130f0     ucrt:api-ms-win-crt-stdio-l1-1-0.dll
 0002:000000f4       __imp____stdio_common_vfprintf 004130f4     ucrt:api-ms-win-crt-stdio-l1-1-0.dll
 0002:000000f8       __imp____p__commode        004130f8     ucrt:api-ms-win-crt-stdio-l1-1-0.dll
 0002:000000fc       __imp__fclose              004130fc     ucrt:api-ms-win-crt-stdio-l1-1-0.dll
 0002:00000100       __imp____stdio_common_vsprintf 00413100     ucrt:api-ms-win-crt-stdio-l1-1-0.dll
 0002:00000104       __imp___set_fmode          00413104     ucrt:api-ms-win-crt-stdio-l1-1-0.dll
 0002:00000108       __imp__fopen               00413108     ucrt:api-ms-win-crt-stdio-l1-1-0.dll
 0002:0000010c       __imp__fread               0041310c     ucrt:api-ms-win-crt-stdio-l1-1-0.dll
 0002:00000110       __imp___fileno             00413110     ucrt:api-ms-win-crt-stdio-l1-1-0.dll
 0002:00000110       __imp__fileno              00413110     ucrt:api-ms-win-crt-stdio-l1-1-0.dll
 0002:00000114       __imp__fflush              00413114     ucrt:api-ms-win-crt-stdio-l1-1-0.dll
 0002:00000118       \177api-ms-win-crt-stdio-l1-1-0_NULL_THUNK_DATA 00413118     ucrt:api-ms-win-crt-stdio-l1-1-0.dll
 0002:0000011c       __imp__strdup              0041311c     ucrt:api-ms-win-crt-string-l1-1-0.dll
 0002:0000011c       __imp___strdup             0041311c     ucrt:api-ms-win-crt-string-l1-1-0.dll
 0002:00000120       __imp__strncat             00413120     ucrt:api-ms-win-crt-string-l1-1-0.dll
 0002:00000124       __imp__strtok              00413124     ucrt:api-ms-win-crt-string-l1-1-0.dll
 0002:00000128       __imp__strcat              00413128     ucrt:api-ms-win-crt-string-l1-1-0.dll
 0002:0000012c       __imp__strcmp              0041312c     ucrt:api-ms-win-crt-string-l1-1-0.dll
 0002:00000130       __imp__strncmp             00413130     ucrt:api-ms-win-crt-string-l1-1-0.dll
 0002:00000134       __imp__strlen              00413134     ucrt:api-ms-win-crt-string-l1-1-0.dll
 0002:00000138       \177api-ms-win-crt-string-l1-1-0_NULL_THUNK_DATA 00413138     ucrt:api-ms-win-crt-string-l1-1-0.dll
 0002:0000013c       __imp___gmtime64           0041313c     ucrt:api-ms-win-crt-time-l1-1-0.dll
 0002:00000140       __imp___time64             00413140     ucrt:api-ms-win-crt-time-l1-1-0.dll
 0002:00000144       \177api-ms-win-crt-time-l1-1-0_NULL_THUNK_DATA 00413144     ucrt:api-ms-win-crt-time-l1-1-0.dll
 0002:00000148       __imp__qsort               00413148     ucrt:api-ms-win-crt-utility-l1-1-0.dll
 0002:0000014c       \177api-ms-win-crt-utility-l1-1-0_NULL_THUNK_DATA 0041314c     ucrt:api-ms-win-crt-utility-l1-1-0.dll
 0002:00000150       ___guard_check_icall_fptr  00413150     MSVCRT:guard_support.obj
 0002:00000154       ___xc_a                    00413154     MSVCRT:initializers.obj
 0002:0000015c       ___xc_z                    0041315c     MSVCRT:initializers.obj
 0002:00000160       ___xi_a                    00413160     MSVCRT:initializers.obj
 0002:0000016c       ___xi_z                    0041316c     MSVCRT:initializers.obj
 0002:00000170       ___xp_a                    00413170     MSVCRT:initializers.obj
 0002:00000174       ___xp_z                    00413174     MSVCRT:initializers.obj
 0002:00000178       ___xt_a                    00413178     MSVCRT:initializers.obj
 0002:0000017c       ___xt_z                    0041317c     MSVCRT:initializers.obj
 0002:00000180       ??_C@_05OJPKCACG@1?43?41@  00413180     compress.obj
 0002:00000188       _deflate_copyright         00413188     deflate.obj
 0002:00000af8       ??_C@_0BD@PJCBIDD@invalid?5block?5type@ 00413af8     infback.obj
 0002:00000b0c       ??_C@_0BN@LGAADGOK@invalid?5stored?5block?5lengths@ 00413b0c     infback.obj
 0002:00000b2c       ??_C@_0CE@GMIGFPBB@too?5many?5length?5or?5distance?5sym@ 00413b2c     infback.obj
 0002:00000b50       ??_C@_0BJ@HDEPPGOH@invalid?5code?5lengths?5set@ 00413b50     infback.obj
 0002:00000b6c       ??_C@_0BK@BMMPFBBH@invalid?5bit?5length?5repeat@ 00413b6c     infback.obj
 0002:00000b88       ??_C@_0CF@DGDMADCD@invalid?5code?5?9?9?5missing?5end?9of?9@ 00413b88     infback.obj
 0002:00000bb0       ??_C@_0BM@IIMGAINC@invalid?5literal?1lengths?5set@ 00413bb0     infback.obj
 0002:00000bcc       ??_C@_0BG@GMDFCBGP@invalid?5distances?5set@ 00413bcc     infback.obj
 0002:00000be4       ??_C@_0BM@FFFLPBBC@invalid?5literal?1length?5code@ 00413be4     infback.obj
 0002:00000c00       ??_C@_0BG@LBKINIKP@invalid?5distance?5code@ 00413c00     infback.obj
 0002:00000c18       ??_C@_0BO@ECPMAOGG@invalid?5distance?5too?5far?5back@ 00413c18     infback.obj
 0002:000014e0       ??_C@_0BH@LIBMMIGA@incorrect?5header?5check@ 004144e0     inflate.obj
 0002:000014f8       ??_C@_0BL@IHKGDAEE@unknown?5compression?5method@ 004144f8     inflate.obj
 0002:00001514       ??_C@_0BE@EMOGCLGO@invalid?5window?5size@ 00414514     inflate.obj
 0002:00001528       ??_C@_0BJ@BLBBCOMO@unknown?5header?5flags?5set@ 00414528     inflate.obj
 0002:00001544       ??_C@_0BE@GONKLEPM@header?5crc?5mismatch@ 00414544     inflate.obj
 0002:00001558       ??_C@_0BF@MEIGEHBE@incorrect?5data?5check@ 00414558     inflate.obj
 0002:00001570       ??_C@_0BH@FGKKJGOC@incorrect?5length?5check@ 00414570     inflate.obj
 0002:00001588       _inflate_copyright         00414588     inftrees.obj
 0002:000016b8       __length_code              004146b8     trees.obj
 0002:000017b8       __dist_code                004147b8     trees.obj
 0002:000049b0       ??_C@_0BA@MOKMMFOD@need?5dictionary@ 004179b0     zutil.obj
 0002:000049c0       ??_C@_0L@FNAOCBOG@stream?5end@ 004179c0     zutil.obj
 0002:000049cb       ??_C@_00CNPNBAHC@@         004179cb     zutil.obj
 0002:000049cc       ??_C@_0L@KIJFAKBJ@file?5error@ 004179cc     zutil.obj
 0002:000049d8       ??_C@_0N@MKKNPMJD@stream?5error@ 004179d8     zutil.obj
 0002:000049e8       ??_C@_0L@HAHMBNLP@data?5error@ 004179e8     zutil.obj
 0002:000049f4       ??_C@_0BE@OGGJBMCE@insufficient?5memory@ 004179f4     zutil.obj
 0002:00004a08       ??_C@_0N@DFPGLBGC@buffer?5error@ 00417a08     zutil.obj
 0002:00004a18       ??_C@_0BF@CJFPCCEG@incompatible?5version@ 00417a18     zutil.obj
 0002:00004a30       _z_errmsg                  00417a30     zutil.obj
 0002:00005418       ??_C@_0P@NFDCFGCL@cp_Utf8_prefix@ 00418418     bands.obj
 0002:00005428       ??_C@_0P@LOHPAGNO@cp_Utf8_suffix@ 00418428     bands.obj
 0002:00005438       ??_C@_0O@IHLLKPBK@cp_Utf8_chars@ 00418438     bands.obj
 0002:00005448       ??_C@_0BD@EOIEJGOP@cp_Utf8_big_suffix@ 00418448     bands.obj
 0002:0000545c       ??_C@_0BC@HDLINKIK@cp_Utf8_big_chars@ 0041845c     bands.obj
 0002:00005470       ??_C@_06IGKKGOEN@cp_Int@   00418470     bands.obj
 0002:00005478       ??_C@_08OBBFNHHD@cp_Float@ 00418478     bands.obj
 0002:00005484       ??_C@_0L@HNFJMOEO@cp_Long_hi@ 00418484     bands.obj
 0002:00005490       ??_C@_0L@CMAKMBBE@cp_Long_lo@ 00418490     bands.obj
 0002:0000549c       ??_C@_0N@CPNNOOPC@cp_Double_hi@ 0041849c     bands.obj
 0002:000054ac       ??_C@_0N@HOIOOBKI@cp_Double_lo@ 004184ac     bands.obj
 0002:000054bc       ??_C@_09HFEHKGNE@cp_String@ 004184bc     bands.obj
 0002:000054c8       ??_C@_08BOENACK@cp_Class@  004184c8     bands.obj
 0002:000054d4       ??_C@_0BC@FENMLAPO@cp_Signature_form@ 004184d4     bands.obj
 0002:000054e8       ??_C@_0BF@MEOEAPGK@cp_Signature_classes@ 004184e8     bands.obj
 0002:00005500       ??_C@_0O@JHMEINNJ@cp_Descr_name@ 00418500     bands.obj
 0002:00005510       ??_C@_0O@DMMHENKJ@cp_Descr_type@ 00418510     bands.obj
 0002:00005520       ??_C@_0P@EEAFDJFH@cp_Field_class@ 00418520     bands.obj
 0002:00005530       ??_C@_0O@FCFAPCDP@cp_Field_desc@ 00418530     bands.obj
 0002:00005540       ??_C@_0BA@LDOOFFKI@cp_Method_class@ 00418540     bands.obj
 0002:00005550       ??_C@_0P@NLGLFAKL@cp_Method_desc@ 00418550     bands.obj
 0002:00005560       ??_C@_0BB@IIGJKIIK@cp_Imethod_class@ 00418560     bands.obj
 0002:00005574       ??_C@_0BA@DCLGLKIL@cp_Imethod_desc@ 00418574     bands.obj
 0002:00005584       ??_C@_0BI@NIJEEAN@cp_MethodHandle_refkind@ 00418584     bands.obj
 0002:0000559c       ??_C@_0BH@NKNCKAEO@cp_MethodHandle_member@ 0041859c     bands.obj
 0002:000055b4       ??_C@_0O@NHPECHNH@cp_MethodType@ 004185b4     bands.obj
 0002:000055c4       ??_C@_0BH@NPCIPIPL@cp_BootstrapMethod_ref@ 004185c4     bands.obj
 0002:000055dc       ??_C@_0BN@DJLEBMBH@cp_BootstrapMethod_arg_count@ 004185dc     bands.obj
 0002:000055fc       ??_C@_0BH@JNPGIEDO@cp_BootstrapMethod_arg@ 004185fc     bands.obj
 0002:00005614       ??_C@_0BG@CIPOMBAC@cp_InvokeDynamic_spec@ 00418614     bands.obj
 0002:0000562c       ??_C@_0BG@IFFCPCPP@cp_InvokeDynamic_desc@ 0041862c     bands.obj
 0002:00005644       ??_C@_0BI@KJJNKCHD@attr_definition_headers@ 00418644     bands.obj
 0002:0000565c       ??_C@_0BF@EEAHHHEA@attr_definition_name@ 0041865c     bands.obj
 0002:00005674       ??_C@_0BH@EKDDDJNL@attr_definition_layout@ 00418674     bands.obj
 0002:0000568c       ??_C@_0O@HJMNFDHJ@ic_this_class@ 0041868c     bands.obj
 0002:0000569c       ??_C@_08CKLAPDFF@ic_flags@ 0041869c     bands.obj
 0002:000056a8       ??_C@_0P@MGLGIOLC@ic_outer_class@ 004186a8     bands.obj
 0002:000056b8       ??_C@_07OPOCOJIH@ic_name@  004186b8     bands.obj
 0002:000056c0       ??_C@_0L@GONOGKKN@class_this@ 004186c0     bands.obj
 0002:000056cc       ??_C@_0M@FMPLOBH@class_super@ 004186cc     bands.obj
 0002:000056d8       ??_C@_0BG@ELABOHHB@class_interface_count@ 004186d8     bands.obj
 0002:000056f0       ??_C@_0BA@GDKGLIFF@class_interface@ 004186f0     bands.obj
 0002:00005700       ??_C@_0BC@GLACLOBG@class_field_count@ 00418700     bands.obj
 0002:00005714       ??_C@_0BD@MFLGOFPO@class_method_count@ 00418714     bands.obj
 0002:00005728       ??_C@_0M@IINMAGFA@field_descr@ 00418728     bands.obj
 0002:00005734       ??_C@_0P@LDBPJHCP@field_flags_hi@ 00418734     bands.obj
 0002:00005744       ??_C@_0P@OCEMJIHF@field_flags_lo@ 00418744     bands.obj
 0002:00005754       ??_C@_0BB@GJGJJLKK@field_attr_count@ 00418754     bands.obj
 0002:00005768       ??_C@_0BD@LLAABMND@field_attr_indexes@ 00418768     bands.obj
 0002:0000577c       ??_C@_0BB@LHINHPHH@field_attr_calls@ 0041877c     bands.obj
 0002:00005790       ??_C@_0BH@NKCAAIDC@field_ConstantValue_KQ@ 00418790     bands.obj
 0002:000057a8       ??_C@_0BD@HMEKDNDB@field_Signature_RS@ 004187a8     bands.obj
 0002:000057bc       ??_C@_0BF@KACJMLOM@field_metadata_bands@ 004187bc     bands.obj
 0002:000057d4       ??_C@_0BB@NIMLDFOB@field_attr_bands@ 004187d4     bands.obj
 0002:000057e8       ??_C@_0N@GLCNNANE@method_descr@ 004187e8     bands.obj
 0002:000057f8       ??_C@_0BA@EIPLIEID@method_flags_hi@ 004187f8     bands.obj
 0002:00005808       ??_C@_0BA@BJKIILNJ@method_flags_lo@ 00418808     bands.obj
 0002:00005818       ??_C@_0BC@OPGFNCHF@method_attr_count@ 00418818     bands.obj
 0002:0000582c       ??_C@_0BE@LCKALKDL@method_attr_indexes@ 0041882c     bands.obj
 0002:00005840       ??_C@_0BC@DBIBDGKI@method_attr_calls@ 00418840     bands.obj
 0002:00005854       ??_C@_0BE@HAIBKECN@method_Exceptions_N@ 00418854     bands.obj
 0002:00005868       ??_C@_0BF@ILMHJLAD@method_Exceptions_RC@ 00418868     bands.obj
 0002:00005880       ??_C@_0BE@HFOKJLNJ@method_Signature_RS@ 00418880     bands.obj
 0002:00005894       ??_C@_0BG@JDLLNHF@method_metadata_bands@ 00418894     bands.obj
 0002:000058ac       ??_C@_0BL@MNBFAABE@method_MethodParameters_NB@ 004188ac     bands.obj
 0002:000058c8       ??_C@_0CB@POGNKHAK@method_MethodParameters_name_RU@ 004188c8     bands.obj
 0002:000058ec       ??_C@_0CA@HDKLJONB@method_MethodParameters_flag_FH@ 004188ec     bands.obj
 0002:0000590c       ??_C@_0BC@FOMHHMDO@method_attr_bands@ 0041890c     bands.obj
 0002:00005920       ??_C@_0P@DNMDIOJK@class_flags_hi@ 00418920     bands.obj
 0002:00005930       ??_C@_0P@GMJAIBMA@class_flags_lo@ 00418930     bands.obj
 0002:00005940       ??_C@_0BB@JELAOHEL@class_attr_count@ 00418940     bands.obj
 0002:00005954       ??_C@_0BD@KFNGBOLA@class_attr_indexes@ 00418954     bands.obj
 0002:00005968       ??_C@_0BB@EKFEADJG@class_attr_calls@ 00418968     bands.obj
 0002:0000597c       ??_C@_0BF@MJNFEGEM@class_SourceFile_RUN@ 0041897c     bands.obj
 0002:00005994       ??_C@_0BJ@CCGEELON@class_EnclosingMethod_RC@ 00418994     bands.obj
 0002:000059b0       ??_C@_0BK@LFCMIOIA@class_EnclosingMethod_RDN@ 004189b0     bands.obj
 0002:000059cc       ??_C@_0BD@GCJMDPFC@class_Signature_RS@ 004189cc     bands.obj
 0002:000059e0       ??_C@_0BF@PHIMHC@class_metadata_bands@ 004189e0     bands.obj
 0002:000059f8       ??_C@_0BF@PGJMDHG@class_InnerClasses_N@ 004189f8     bands.obj
 0002:00005a10       ??_C@_0BG@HHABPLBI@class_InnerClasses_RC@ 00418a10     bands.obj
 0002:00005a28       ??_C@_0BF@MHLAEJHO@class_InnerClasses_F@ 00418a28     bands.obj
 0002:00005a40       ??_C@_0BN@FANFKEPF@class_InnerClasses_outer_RCN@ 00418a40     bands.obj
 0002:00005a60       ??_C@_0BM@CHKHAMMI@class_InnerClasses_name_RUN@ 00418a60     bands.obj
 0002:00005a7c       ??_C@_0CA@LBNJCLO@class_ClassFile_version_minor_H@ 00418a7c     bands.obj
 0002:00005a9c       ??_C@_0CA@KDGDJOMP@class_ClassFile_version_major_H@ 00418a9c     bands.obj
 0002:00005abc       ??_C@_0BB@CFBCEJAA@class_attr_bands@ 00418abc     bands.obj
 0002:00005ad0       ??_C@_0N@EJFJBMLJ@code_headers@ 00418ad0     bands.obj
 0002:00005ae0       ??_C@_0P@DPBEANCA@code_max_stack@ 00418ae0     bands.obj
 0002:00005af0       ??_C@_0BD@OBGMDNFJ@code_max_na_locals@ 00418af0     bands.obj
 0002:00005b04       ??_C@_0BD@OMMDBBC@code_handler_count@ 00418b04     bands.obj
 0002:00005b18       ??_C@_0BF@NAEEIJON@code_handler_start_P@ 00418b18     bands.obj
 0002:00005b30       ??_C@_0BE@GIJMHOG@code_handler_end_PO@ 00418b30     bands.obj
 0002:00005b44       ??_C@_0BG@GJGNOMGM@code_handler_catch_PO@ 00418b44     bands.obj
 0002:00005b5c       ??_C@_0BH@ECFPKFHF@code_handler_class_RCN@ 00418b5c     bands.obj
 0002:00005b74       ??_C@_0O@PKFJGJJN@code_flags_hi@ 00418b74     bands.obj
 0002:00005b84       ??_C@_0O@KLAKGGMH@code_flags_lo@ 00418b84     bands.obj
 0002:00005b94       ??_C@_0BA@OFJPMBMN@code_attr_count@ 00418b94     bands.obj
 0002:00005ba4       ??_C@_0BC@BKACNFKP@code_attr_indexes@ 00418ba4     bands.obj
 0002:00005bb8       ??_C@_0BA@DLHLCFBA@code_attr_calls@ 00418bb8     bands.obj
 0002:00005bc8       ??_C@_0BF@FNGGAIBD@code_StackMapTable_N@ 00418bc8     bands.obj
 0002:00005be0       ??_C@_0BL@IJLKAPMG@code_StackMapTable_frame_T@ 00418be0     bands.obj
 0002:00005bfc       ??_C@_0BL@FLGOBHFL@code_StackMapTable_local_N@ 00418bfc     bands.obj
 0002:00005c18       ??_C@_0BL@DBPDDGDK@code_StackMapTable_stack_N@ 00418c18     bands.obj
 0002:00005c34       ??_C@_0BK@HMGLLHPP@code_StackMapTable_offset@ 00418c34     bands.obj
 0002:00005c50       ??_C@_0BF@ONELPCMI@code_StackMapTable_T@ 00418c50     bands.obj
 0002:00005c68       ??_C@_0BG@EKILGBAE@code_StackMapTable_RC@ 00418c68     bands.obj
 0002:00005c80       ??_C@_0BF@IJCHDHMM@code_StackMapTable_P@ 00418c80     bands.obj
 0002:00005c98       ??_C@_0BH@EMJOIADC@code_LineNumberTable_N@ 00418c98     bands.obj
 0002:00005cb0       ??_C@_0BL@BODGMFAF@code_LineNumberTable_bci_P@ 00418cb0     bands.obj
 0002:00005ccc       ??_C@_0BK@KMDHKKJP@code_LineNumberTable_line@ 00418ccc     bands.obj
 0002:00005ce8       ??_C@_0BK@EAEINMEG@code_LocalVariableTable_N@ 00418ce8     bands.obj
 0002:00005d04       ??_C@_0BO@EBBJALKI@code_LocalVariableTable_bci_P@ 00418d04     bands.obj
 0002:00005d24       ??_C@_0BP@JIPNBFGM@code_LocalVariableTable_span_O@ 00418d24     bands.obj
 0002:00005d44       ??_C@_0CA@LBKLALLO@code_LocalVariableTable_name_RU@ 00418d44     bands.obj
 0002:00005d64       ??_C@_0CA@OBPDECDH@code_LocalVariableTable_type_RS@ 00418d64     bands.obj
 0002:00005d84       ??_C@_0BN@BAELGOA@code_LocalVariableTable_slot@ 00418d84     bands.obj
 0002:00005da4       ??_C@_0BO@HHCIFDPC@code_LocalVariableTypeTable_N@ 00418da4     bands.obj
 0002:00005dc4       ??_C@_0CC@OECAEAHA@code_LocalVariableTypeTable_bci@ 00418dc4     bands.obj
 0002:00005de8       ??_C@_0CD@BAFAHGMB@code_LocalVariableTypeTable_spa@ 00418de8     bands.obj
 0002:00005e0c       ??_C@_0CE@BJEEHJII@code_LocalVariableTypeTable_nam@ 00418e0c     bands.obj
 0002:00005e30       ??_C@_0CE@EJBMDAAB@code_LocalVariableTypeTable_typ@ 00418e30     bands.obj
 0002:00005e54       ??_C@_0CB@DCPKAFMH@code_LocalVariableTypeTable_slo@ 00418e54     bands.obj
 0002:00005e78       ??_C@_0BA@FEDNGPIG@code_attr_bands@ 00418e78     bands.obj
 0002:00005e88       ??_C@_08ILNCKCLH@bc_codes@ 00418e88     bands.obj
 0002:00005e94       ??_C@_0O@NHDHOKJ@bc_case_count@ 00418e94     bands.obj
 0002:00005ea4       ??_C@_0O@IPODCEHE@bc_case_value@ 00418ea4     bands.obj
 0002:00005eb4       ??_C@_07PBCCPPFP@bc_byte@  00418eb4     bands.obj
 0002:00005ebc       ??_C@_08LLANNIAP@bc_short@ 00418ebc     bands.obj
 0002:00005ec8       ??_C@_08CNAAIOJJ@bc_local@ 00418ec8     bands.obj
 0002:00005ed4       ??_C@_08CNIFPPEB@bc_label@ 00418ed4     bands.obj
 0002:00005ee0       ??_C@_09LMIAJDCB@bc_intref@ 00418ee0     bands.obj
 0002:00005eec       ??_C@_0M@GHNOKACA@bc_floatref@ 00418eec     bands.obj
 0002:00005ef8       ??_C@_0L@FECALBEM@bc_longref@ 00418ef8     bands.obj
 0002:00005f04       ??_C@_0N@BLIIPDNE@bc_doubleref@ 00418f04     bands.obj
 0002:00005f14       ??_C@_0N@MPKFBKGB@bc_stringref@ 00418f14     bands.obj
 0002:00005f24       ??_C@_0BE@JPNLPCGD@bc_loadablevalueref@ 00418f24     bands.obj
 0002:00005f38       ??_C@_0M@IBEIOBLC@bc_classref@ 00418f38     bands.obj
 0002:00005f44       ??_C@_0M@FHDAHFFG@bc_fieldref@ 00418f44     bands.obj
 0002:00005f50       ??_C@_0N@KBJNFGEO@bc_methodref@ 00418f50     bands.obj
 0002:00005f60       ??_C@_0O@BOILABNA@bc_imethodref@ 00418f60     bands.obj
 0002:00005f70       ??_C@_0L@MEPMLOBJ@bc_indyref@ 00418f70     bands.obj
 0002:00005f7c       ??_C@_0N@CGLIFEKH@bc_thisfield@ 00418f7c     bands.obj
 0002:00005f8c       ??_C@_0O@NMPFAKNK@bc_superfield@ 00418f8c     bands.obj
 0002:00005f9c       ??_C@_0O@OCHHHCLJ@bc_thismethod@ 00418f9c     bands.obj
 0002:00005fac       ??_C@_0P@MMDJDCGG@bc_supermethod@ 00418fac     bands.obj
 0002:00005fbc       ??_C@_0L@IAPCGJHG@bc_initref@ 00418fbc     bands.obj
 0002:00005fc8       ??_C@_09BGKIKDIC@bc_escref@ 00418fc8     bands.obj
 0002:00005fd4       ??_C@_0O@LHNEEOML@bc_escrefsize@ 00418fd4     bands.obj
 0002:00005fe4       ??_C@_0L@HJKABJFB@bc_escsize@ 00418fe4     bands.obj
 0002:00005ff0       ??_C@_0L@HOKHNNPG@bc_escbyte@ 00418ff0     bands.obj
 0002:00005ffc       ??_C@_09GOEDCGAO@file_name@ 00418ffc     bands.obj
 0002:00006008       ??_C@_0N@INICLDFG@file_size_hi@ 00419008     bands.obj
 0002:00006018       ??_C@_0N@NMNBLMAM@file_size_lo@ 00419018     bands.obj
 0002:00006028       ??_C@_0N@JMABFCDG@file_modtime@ 00419028     bands.obj
 0002:00006038       ??_C@_0N@OPKBLMJG@file_options@ 00419038     bands.obj
 0002:00006048       ??_C@_08FPGGDHDD@no?5index@ 00419048     bands.obj
 0002:00006054       ??_C@_08CHILEFNK@null?5ref@ 00419054     bands.obj
 0002:00006060       ??_C@_07MLPLAPLE@bad?5ref@ 00419060     bands.obj
 0002:00006068       ??_C@_0BC@CJBOIHCG@overflow?5detected@ 00419068     bands.obj
 0002:0000607c       ??_C@_0BJ@CALEAGEE@Native?5allocation?5failed@ 0041907c     bytes.obj
 0002:000060ac       ??_C@_0BA@MMOCMGFH@bad?5value?5count@ 004190ac     coding.obj
 0002:000060bc       ??_C@_0L@FLIJCFOD@bad?5coding@ 004190bc     coding.obj
 0002:000060c8       ??_C@_0BE@IIPOPKNG@illegal?5arb?4?5coding@ 004190c8     coding.obj
 0002:000060dc       ??_C@_0BF@OEPDPLDN@illegal?5run?5encoding@ 004190dc     coding.obj
 0002:000060f4       ??_C@_0BM@FJMGNNPG@illegal?5nested?5run?5encoding@ 004190f4     coding.obj
 0002:00006110       ??_C@_0BF@JOAAKECG@illegal?5pop?5encoding@ 00419110     coding.obj
 0002:00006128       ??_C@_0BM@CDDFICON@illegal?5nested?5pop?5encoding@ 00419128     coding.obj
 0002:00006144       ??_C@_0BG@HLIJPJNL@pop?4L?5value?5too?5small@ 00419144     coding.obj
 0002:0000615c       ??_C@_0BH@OCEIAIEJ@pop?5token?5out?5of?5range@ 0041915c     coding.obj
 0002:00006174       ??_C@_0CA@HBCNKKJO@bad?5meta?9coding?5for?5empty?5pop?1U@ 00419174     coding.obj
 0002:00006194       ??_C@_0BA@DAENMACF@bad?5meta?9coding@ 00419194     coding.obj
 0002:000061c0       ??_C@_02DPKJAMEF@?$CFd@    004191c0     main.obj
 0002:000061c4       ??_C@_09NIKIINED@unpack200@ 004191c4     main.obj
 0002:000061d0       ??_C@_0DM@OIAPDBBH@Usage?3?5?5?$CFs?5?$FL?9opt?4?4?4?5?$HM?5?9?9option?$DN@ 004191d0     main.obj
 0002:00006210       ??_C@_0CHL@BBGKGDMF@?6Unpacking?5Options?6?5?5?9H?$HLh?$HN?0?5?9?9d@ 00419210     main.obj
 0002:0000648c       ??_C@_0CJ@KKLFNMLF@?$CIFor?5more?5information?0?5run?5?$CFs?5?9@ 0041948c     main.obj
 0002:000064b8       ??_C@_0BA@OCMGBEIP@UNPACK200_FLAGS@ 004194b8     main.obj
 0002:000064c8       ??_C@_03CLFDNPKK@?6?7?5@   004194c8     main.obj
 0002:000064cc       ??_C@_0CB@HAIPLNAM@?9XDsuppress?9tool?9removal?9messag@ 004194cc     main.obj
 0002:000064f0       ??_C@_0P@BDFHEJH@Hdeflate?9hint?$DN@ 004194f0     main.obj
 0002:00006500       ??_C@_08KBJOIMAC@vverbose@ 00419500     main.obj
 0002:0000650c       ??_C@_06JKKBEHHF@qquiet@   0041950c     main.obj
 0002:00006514       ??_C@_0BC@PMPEJJOP@rremove?9pack?9file@ 00419514     main.obj
 0002:00006528       ??_C@_0L@ONHIOBCM@llog?9file?$DN@ 00419528     main.obj
 0002:00006534       ??_C@_08KNEMGMJA@Vversion@ 00419534     main.obj
 0002:00006540       ??_C@_05GBNCKDGE@hhelp@    00419540     main.obj
 0002:00006548       ??_C@_0FL@LHNBJCPB@?6Warning?3?5The?5?$CFs?5tool?5is?5deprec@ 00419548     main.obj
 0002:000065a4       ??_C@_0BE@DAFJFMML@unpack?4deflate?4hint@ 004195a4     main.obj
 0002:000065b8       ??_C@_01HIHLOKLC@1@        004195b8     main.obj
 0002:000065bc       ??_C@_0DC@KGJOKPLE@com?4sun?4java?4util?4jar?4pack?4unpa@ 004195bc     main.obj
 0002:000065f0       ??_C@_0P@BNKJLCIA@?$CFs?5version?5?$CFs?6@ 004195f0     main.obj
 0002:00006600       ??_C@_0BH@ODCNNNPJ@?5in?5$?$HLUNPACK200_FLAGS?$HN@ 00419600     main.obj
 0002:00006618       ??_C@_0BN@OPJBPAAA@Missing?5option?5string?$CFs?3?5?$CFs?6@ 00419618     main.obj
 0002:00006638       ??_C@_0BN@OCHJBIAD@Unrecognized?5argument?$CFs?3?5?$CFs?6@ 00419638     main.obj
 0002:00006658       ??_C@_0CD@CEMFBAGC@com?4sun?4java?4util?4jar?4pack?4verb@ 00419658     main.obj
 0002:0000667c       ??_C@_0CL@JFLJFCLE@com?4sun?4java?4util?4jar?4pack?4unpa@ 0041967c     main.obj
 0002:000066a8       ??_C@_0BJ@LIHJOOPB@Unpacking?5from?5?$CFs?5to?5?$CFs?6@ 004196a8     main.obj
 0002:000066c4       ??_C@_01JOAMLHOP@?9@       004196c4     main.obj
 0002:000066c8       ??_C@_02JDPG@rb@           004196c8     main.obj
 0002:000066cc       ??_C@_0CG@FKHOAOGE@Error?3?5Could?5not?5open?5input?5fil@ 004196cc     main.obj
 0002:000066f4       ??_C@_0CC@NBFDMLEM@garbage?5after?5end?5of?5pack?5archi@ 004196f4     main.obj
 0002:00006718       ??_C@_0L@DCCGFMBN@Error?3?5?$CFs?6@ 00419718     main.obj
 0002:00006724       ??_C@_0CD@KGGFLFGJ@unpacker?5completed?5with?5status?$DN@ 00419724     main.obj
 0002:00006778       ??_C@_0BC@DHBHLEDC@bad?5utf8?5encoding@ 00419778     unpack.obj
 0002:0000678c       ??_C@_08MPEBFEBH@bad?5data@ 0041978c     unpack.obj
 0002:00006798       ??_C@_0BI@MCADJHPK@missing?5class?5reference@ 00419798     unpack.obj
 0002:000067b0       ??_C@_0BJ@DINDGABB@Internal?5buffer?5overflow@ 004197b0     unpack.obj
 0002:000067cc       ??_C@_0BE@NBGJPKOJ@too?5much?5read?9ahead@ 004197cc     unpack.obj
 0002:000067e0       ??_C@_0CB@MBENKFPE@EOF?5reading?5archive?5magic?5numbe@ 004197e0     unpack.obj
 0002:00006804       ??_C@_0M@HDHEHMIJ@Copy?9mode?4?6@ 00419804     unpack.obj
 0002:00006810       ??_C@_0GN@MIAOKBBJ@?$EACorrupted?5pack?5file?3?5magic?1ver@ 00419810     unpack.obj
 0002:00006880       ??_C@_0DJ@EOFNCHGA@Format?5bits?5for?5Java?57?5must?5be?5@ 00419880     unpack.obj
 0002:000068bc       ??_C@_0DH@PDJEDCEA@High?5archive?5option?5bits?5are?5re@ 004198bc     unpack.obj
 0002:000068f4       ??_C@_0BP@CKGMAJKP@EOF?5reading?5fixed?5input?5buffer@ 004198f4     unpack.obj
 0002:00006914       ??_C@_0BI@EDJMKDIH@impossible?5archive?5size@ 00419914     unpack.obj
 0002:0000692c       ??_C@_0DE@HNNKIDEL@cannot?5allocate?5large?5input?5buf@ 0041992c     unpack.obj
 0002:00006960       ??_C@_0BL@KOJPDLNM@EOF?5reading?5archive?5header@ 00419960     unpack.obj
 0002:0000697c       ??_C@_0BJ@HODOOMDO@EOF?5reading?5band?5headers@ 0041997c     unpack.obj
 0002:00006998       ??_C@_0DD@FJENCPEO@A?5total?5of?5?$CFlld?5bytes?5were?5read@ 00419998     unpack.obj
 0002:000069cc       ??_C@_0DC@HIEHJDF@A?5total?5of?5?$CFlld?5file?5content?5by@ 004199cc     unpack.obj
 0002:00006a00       ??_C@_0EH@BADKEGGH@A?5total?5of?5?$CFd?5files?5?$CIof?5which?5?$CF@ 00419a00     unpack.obj
 0002:00006a48       ??_C@_0DB@HCOAOCOI@archive?5too?5large?3?5?5constant?5po@ 00419a48     unpack.obj
 0002:00006a7c       ??_C@_0BA@BMKLBFBL@bad?5utf8?5suffix@ 00419a7c     unpack.obj
 0002:00006a8c       ??_C@_0BA@HHOGEFOO@bad?5utf8?5prefix@ 00419a8c     unpack.obj
 0002:00006a9c       ??_C@_0BF@HNBIPEII@utf8?5prefix?5overflow@ 00419a9c     unpack.obj
 0002:00006ab4       ??_C@_0BE@INMEHPDO@unexpected?5band?5?$CFs?6@ 00419ab4     unpack.obj
 0002:00006ac8       ??_C@_0BKA@JMJPKLFN@01?$AASignature?$AADeprecated?$AARuntime@ 00419ac8     unpack.obj
 0002:00006c68       ??_C@_0BK@NOGBJPAL@attribute?5index?5too?5large@ 00419c68     unpack.obj
 0002:00006c84       ??_C@_0BK@OFNJKMED@redefined?5attribute?5index@ 00419c84     unpack.obj
 0002:00006ca0       ??_C@_0BJ@OGDEGNBN@garbage?5at?5end?5of?5layout@ 00419ca0     unpack.obj
 0002:00006cbc       ??_C@_0BN@NJCEKHIO@garbage?5mixed?5with?5callables@ 00419cbc     unpack.obj
 0002:00006cdc       ??_C@_0BD@BJONMNHI@bad?5call?5in?5layout@ 00419cdc     unpack.obj
 0002:00006cf0       ??_C@_0BD@EOHIHJFP@bad?5layout?5element@ 00419cf0     unpack.obj
 0002:00006d04       ??_C@_0BK@CHPLBKBJ@missing?5numeral?5in?5layout@ 00419d04     unpack.obj
 0002:00006d20       ??_C@_0BB@FJJKEHGJ@numeral?5overflow@ 00419d20     unpack.obj
 0002:00006d34       ??_C@_0P@HDHNKEAB@bad?5union?5case@ 00419d34     unpack.obj
 0002:00006d44       ??_C@_0DD@PGOJPNFL@bad?5range?5in?5union?5case?5label?5?$CI@ 00419d44     unpack.obj
 0002:00006d78       ??_C@_0BO@JELFCPB@bad?5range?5in?5union?5case?5label@ 00419d78     unpack.obj
 0002:00006d98       ??_C@_0P@KBKJHJBF@bad?5case?5label@ 00419d98     unpack.obj
 0002:00006da8       ??_C@_0P@MNJPOPJO@bad?5call?5label@ 00419da8     unpack.obj
 0002:00006db8       ??_C@_0BF@ILAEDGAO@bad?5reference?5layout@ 00419db8     unpack.obj
 0002:00006dd0       ??_C@_0BE@NGGDBALG@bad?5nested?5callable@ 00419dd0     unpack.obj
 0002:00006de4       ??_C@_0L@FLEMDFJG@bad?5layout@ 00419de4     unpack.obj
 0002:00006df0       ??_C@_0JK@BMMFGJDP@?$FLNB?$FL?$CI1?$CJ?$FN?$FN?$FLNH?$FL?$CI1?$CJ?$FN?$FN?$FLRSHNH?$FLRUH?$CI1?$CJ@ 00419df0     unpack.obj
 0002:00006e8c       ??_C@_09MAEOCCFN@?$FLNB?$FL?$CI1?$CJ?$FN?$FN@ 00419e8c     unpack.obj
 0002:00006e98       ??_C@_0CC@PCCOCALL@?$FLNB?$FL?$CI1?$CJ?$FN?$FN?$FLNH?$FL?$CI1?$CJ?$FN?$FN?$FLRSHNH?$FLRUH?$CI1?$CJ@ 00419e98     unpack.obj
 0002:00006ec0       ??_C@_0BBL@GCIMMLOG@?$FLNH?$FL?$CI1?$CJ?$CI2?$CJ?$CI3?$CJ?$FN?$FN?$FLTB?$CI0?01?$CJ?$FLB?$FN?$CI16?$CJ?$FL@ 00419ec0     unpack.obj
 0002:00006fdc       ??_C@_0BK@CIMGHPDJ@RuntimeVisibleAnnotations@ 00419fdc     unpack.obj
 0002:00006ff8       ??_C@_0BM@BNNGFNMF@RuntimeInvisibleAnnotations@ 00419ff8     unpack.obj
 0002:00007014       ??_C@_0CD@ONLIBICP@RuntimeVisibleParameterAnnotati@ 0041a014     unpack.obj
 0002:00007038       ??_C@_0CF@BFEAEHFK@RuntimeInvisibleParameterAnnota@ 0041a038     unpack.obj
 0002:00007060       ??_C@_0BC@DAGIEPHG@AnnotationDefault@ 0041a060     unpack.obj
 0002:00007074       ??_C@_0BO@IJLELCEA@RuntimeVisibleTypeAnnotations@ 0041a074     unpack.obj
 0002:00007094       ??_C@_0CA@GCLMFPKD@RuntimeInvisibleTypeAnnotations@ 0041a094     unpack.obj
 0002:000070b4       ??_C@_0BG@FDJMCAOP@identical?5inner?5class@ 0041a0b4     unpack.obj
 0002:000070cc       ??_C@_0BN@GFADPNEE@undefined?5attribute?5flag?5bit@ 0041a0cc     unpack.obj
 0002:000070ec       ??_C@_0BO@CMGKNLIA@attribute?5index?5out?5of?5bounds@ 0041a0ec     unpack.obj
 0002:0000710c       ??_C@_0DH@OHIKFIJI@undefined?5StackMapTable?5attribu@ 0041a10c     unpack.obj
 0002:00007144       ??_C@_0CL@CLGKHLIF@layout_definition?5pointer?5must?5@ 0041a144     unpack.obj
 0002:00007170       ??_C@_0CE@NENNCDNJ@putlayout?3?5unexpected?5NULL?5for?5@ 0041a170     unpack.obj
 0002:00007194       ??_C@_0BB@HNCAJEIE@cp?5utf8?5overflow@ 0041a194     unpack.obj
 0002:000071a8       ??_C@_0BC@IJJDHGHN@cp?5class?5overflow@ 0041a1a8     unpack.obj
 0002:000071bc       ??_C@_0DE@FNJPLIMN@com?4sun?4java?4util?4jar?4pack?4unpa@ 0041a1bc     unpack.obj
 0002:000071f0       ??_C@_04LKOEDJLC@keep@     0041a1f0     unpack.obj
 0002:000071f8       ??_C@_0CJ@LFNCLCEP@com?4sun?4java?4util?4jar?4pack?4verb@ 0041a1f8     unpack.obj
 0002:00007224       ??_C@_03CGLHMDPP@now@      0041a224     unpack.obj
 0002:00007228       ??_C@_0DL@GFEANCIP@After?5segment?5?$CFd?0?5?$CFlld?5bytes?5re@ 0041a228     unpack.obj
 0002:00007268       ??_C@_0EJ@CMEPGJEN@After?5segment?5?$CFd?0?5?$CFd?5files?5?$CIof?5@ 0041a268     unpack.obj
 0002:000072b4       ??_C@_01LKDEMHDF@s@        0041a2b4     unpack.obj
 0002:000072b8       ??_C@_0DH@GNBHDKCB@After?5segment?5?$CFd?0?5?$CFd?5segment?$CFs?5@ 0041a2b8     unpack.obj
 0002:000072f0       ??_C@_09GHCKAPML@?$CInot?5set?$CJ@ 0041a2f0     unpack.obj
 0002:000072fc       ??_C@_06BAKFFEGN@?$CFs?$DN?$CFs?6@ 0041a2fc     unpack.obj
 0002:00007304       ??_C@_0BB@MNFIFPBF@bad?5KQ?5reference@ 0041a304     unpack.obj
 0002:00007318       ??_C@_0L@PDBBHOGB@bad?5bcimap@ 0041a318     unpack.obj
 0002:00007324       ??_C@_0BM@GPDDEOEP@too?5many?5InnerClasses?5attrs@ 0041a324     unpack.obj
 0002:00007340       ??_C@_05PBJILJE@?4java@    0041a340     unpack.obj
 0002:00007348       ??_C@_0BB@MICPNADP@bad?5layout?5index@ 0041a348     unpack.obj
 0002:0000735c       ??_C@_0BE@BKLBLMJK@bad?5attribute?5index@ 0041a35c     unpack.obj
 0002:00007370       ??_C@_0BN@CLDGGNCI@bad?5reference?5to?5inner?5class@ 0041a370     unpack.obj
 0002:00007390       ??_C@_0P@DHEBFDOP@Internal?5error@ 0041a390     unpack.obj
 0002:000073a0       ??_C@_0CC@IOEIADGN@archive?5header?5had?5incorrect?5si@ 0041a3a0     unpack.obj
 0002:000073c4       ??_C@_0BM@NDDMOHPH@class?5file?5size?5transmitted@ 0041a3c4     unpack.obj
 0002:000073e0       ??_C@_06POIMOJKC@?4class@  0041a3e0     unpack.obj
 0002:000073e8       ??_C@_0BI@CDCINJGA@resource?5file?5too?5large@ 0041a3e8     unpack.obj
 0002:00007400       ??_C@_0BK@NJPACPAH@EOF?5reading?5resource?5file@ 0041a400     unpack.obj
 0002:0000741c       ??_C@_0BJ@NEMIFNOC@Wrote?5?$CFlld?5bytes?5to?3?5?$CFs?6@ 0041a41c     unpack.obj
 0002:00007438       ??_C@_02DPNLHKJD@a?$CL@    0041a438     unpack.obj
 0002:0000743c       ??_C@_0BK@NDLGHGBM@Can?5not?5open?5log?5file?5?$CFs?6@ 0041a43c     unpack.obj
 0002:00007458       ??_C@_0BI@CELHNJPG@error?5unpacking?5archive@ 0041a458     unpack.obj
 0002:00007470       ??_C@_03OFAPEBGM@?$CFs?6@  0041a470     unpack.obj
 0002:00007480       __xmm@00000000000000ab00000001000000aa 0041a480     unpack.obj
 0002:00007490       __xmm@00000001000000a00000000700000096 0041a490     unpack.obj
 0002:000074a0       ??_C@_0CE@HLJAOJEP@corrupt?5pack?5file?5or?5internal?5e@ 0041a4a0     utils.obj
 0002:000074c4       ??_C@_0BF@JFFKOPFD@Error?3?5unpacker?3?5?$CFs?6@ 0041a4c4     utils.obj
 0002:000074dc       ??_C@_0CG@HFNCMKIN@Error?3?5unpacker?3?5no?5current?5ins@ 0041a4dc     utils.obj
 0002:00007510       ??_C@_0CL@EKHPJDGB@Error?3?5write?5on?5output?5file?5fai@ 0041a510     zip.obj
 0002:0000753c       ??_C@_02GMLFBBN@wb@        0041a53c     zip.obj
 0002:00007540       ??_C@_0CE@COMJCOPK@Error?3?5Could?5not?5open?5jar?5file?3@ 0041a540     zip.obj
 0002:00007564       ??_C@_0CO@DCPNMPAF@Error?3?5gmtime?5failure?0?5invalid?5@ 0041a564     zip.obj
 0002:00007594       ??_C@_0BG@NMMFCDCO@error?5inflating?5input@ 0041a594     zip.obj
 0002:000075ac       ??_C@_0CL@NMECEKOA@garbage?5after?5end?5of?5deflated?5i@ 0041a5ac     zip.obj
 0002:000075d8       ??_C@_0DL@PJJNLKFP@Error?3reading?5CRC?5information?5o@ 0041a5d8     zip.obj
 0002:00007614       ??_C@_0DH@LPFNBMGH@Error?3reading?5file?5length?5on?5in@ 0041a614     zip.obj
 0002:0000764c       ??_C@_0CE@EBLNOIJH@CRC?5error?0?5invalid?5compressed?5d@ 0041a64c     zip.obj
 0002:00007670       ??_C@_0BE@BDJJEDBE@cannot?5create?5input@ 0041a670     zip.obj
 0002:00007684       ??_C@_0BE@BMGPHILO@short?5stream?5header@ 0041a684     zip.obj
 0002:00007710       __load_config_used         0041a710     MSVCRT:loadcfg.obj
 0002:000077b0       ___safe_se_handler_table   0041a7b0     <linker-defined>
 0002:00007a78       ___rtc_iaa                 0041aa78     MSVCRT:initsect.obj
 0002:00007a7c       ___rtc_izz                 0041aa7c     MSVCRT:initsect.obj
 0002:00007a80       ___rtc_taa                 0041aa80     MSVCRT:initsect.obj
 0002:00007a84       ___rtc_tzz                 0041aa84     MSVCRT:initsect.obj
 0002:00007b18       __IMPORT_DESCRIPTOR_KERNEL32 0041ab18     kernel32:KERNEL32.dll
 0002:00007b2c       __IMPORT_DESCRIPTOR_VCRUNTIME140 0041ab2c     vcruntime:VCRUNTIME140.dll
 0002:00007b40       __IMPORT_DESCRIPTOR_api-ms-win-crt-heap-l1-1-0 0041ab40     ucrt:api-ms-win-crt-heap-l1-1-0.dll
 0002:00007b54       __IMPORT_DESCRIPTOR_api-ms-win-crt-stdio-l1-1-0 0041ab54     ucrt:api-ms-win-crt-stdio-l1-1-0.dll
 0002:00007b68       __IMPORT_DESCRIPTOR_api-ms-win-crt-filesystem-l1-1-0 0041ab68     ucrt:api-ms-win-crt-filesystem-l1-1-0.dll
 0002:00007b7c       __IMPORT_DESCRIPTOR_api-ms-win-crt-runtime-l1-1-0 0041ab7c     ucrt:api-ms-win-crt-runtime-l1-1-0.dll
 0002:00007b90       __IMPORT_DESCRIPTOR_api-ms-win-crt-string-l1-1-0 0041ab90     ucrt:api-ms-win-crt-string-l1-1-0.dll
 0002:00007ba4       __IMPORT_DESCRIPTOR_api-ms-win-crt-environment-l1-1-0 0041aba4     ucrt:api-ms-win-crt-environment-l1-1-0.dll
 0002:00007bb8       __IMPORT_DESCRIPTOR_api-ms-win-crt-utility-l1-1-0 0041abb8     ucrt:api-ms-win-crt-utility-l1-1-0.dll
 0002:00007bcc       __IMPORT_DESCRIPTOR_api-ms-win-crt-convert-l1-1-0 0041abcc     ucrt:api-ms-win-crt-convert-l1-1-0.dll
 0002:00007be0       __IMPORT_DESCRIPTOR_api-ms-win-crt-time-l1-1-0 0041abe0     ucrt:api-ms-win-crt-time-l1-1-0.dll
 0002:00007bf4       __IMPORT_DESCRIPTOR_api-ms-win-crt-math-l1-1-0 0041abf4     ucrt:api-ms-win-crt-math-l1-1-0.dll
 0002:00007c08       __IMPORT_DESCRIPTOR_api-ms-win-crt-locale-l1-1-0 0041ac08     ucrt:api-ms-win-crt-locale-l1-1-0.dll
 0002:00007c1c       __NULL_IMPORT_DESCRIPTOR   0041ac1c     kernel32:KERNEL32.dll
 0003:00000000       ?basic_codings@@3PAUcoding@@A 0041c000     coding.obj
 0003:00000b30       ___security_cookie_complement 0041cb30     MSVCRT:gs_cookie.obj
 0003:00000b34       ___security_cookie         0041cb34     MSVCRT:gs_cookie.obj
 0003:00000b40       ___scrt_native_dllmain_reason 0041cb40     MSVCRT:utility.obj
 0003:00000b44       ___scrt_default_matherr    0041cb44     MSVCRT:matherr.obj
 0003:00000b50       ___isa_enabled             0041cb50     MSVCRT:cpu_disp.obj
 0003:00000b54       ___scrt_ucrt_dll_is_in_use 0041cb54     MSVCRT:ucrt_stubs.obj
 0003:00000f5c       ?non_mt_current@unpacker@@2PAU1@A 0041cf5c     main.obj
 0003:00000f68       ?_OptionsStorage@?1??__local_stdio_printf_options@@9@4_KA 0041cf68     main.obj
 0003:00001294       ___scrt_current_native_startup_state 0041d294     MSVCRT:utility.obj
 0003:00001298       ___scrt_native_startup_lock 0041d298     MSVCRT:utility.obj
 0003:000012b8       ?__type_info_root_node@@3U__type_info_node@@A 0041d2b8     MSVCRT:tncleanup.obj
 0003:000012c0       ?_OptionsStorage@?1??__local_stdio_scanf_options@@9@4_KA 0041d2c0     MSVCRT:default_local_stdio_options.obj
 0003:000012c8       ___scrt_debugger_hook_flag 0041d2c8     MSVCRT:utility_desktop.obj
 0003:000012cc       ___isa_available           0041d2cc     MSVCRT:cpu_disp.obj
 0003:000012d0       ___favor                   0041d2d0     MSVCRT:cpu_disp.obj
 0003:000012d4       ___dyn_tls_dtor_callback   0041d2d4     <common>
 0003:000012d8       ___dyn_tls_init_callback   0041d2d8     <common>

 entry point at        0001:00011206

 Static symbols

 0000:fffe0000       .debug$S                   00400000     kernel32:KERNEL32.dll
 0000:fffe0000       .debug$S                   00400000     kernel32:KERNEL32.dll
 0000:fffe0000       .debug$S                   00400000     kernel32:KERNEL32.dll
 0000:fffe0000       .debug$S                   00400000     kernel32:KERNEL32.dll
 0000:fffe0000       .debug$S                   00400000     kernel32:KERNEL32.dll
 0000:fffe0000       .debug$S                   00400000     kernel32:KERNEL32.dll
 0000:fffe0000       .debug$S                   00400000     unpack200.exp
 0000:fffe0000       .debug$S                   00400000     kernel32:KERNEL32.dll
 0000:fffe0000       .debug$S                   00400000     kernel32:KERNEL32.dll
 0000:fffe0000       .debug$S                   00400000     vcruntime:VCRUNTIME140.dll
 0000:fffe0000       .debug$S                   00400000     kernel32:KERNEL32.dll
 0000:fffe0000       .debug$S                   00400000     kernel32:KERNEL32.dll
 0000:fffe0000       .debug$S                   00400000     kernel32:KERNEL32.dll
 0000:fffe0000       .debug$S                   00400000     kernel32:KERNEL32.dll
 0000:fffe0000       .debug$S                   00400000     kernel32:KERNEL32.dll
 0000:fffe0000       .debug$S                   00400000     vcruntime:VCRUNTIME140.dll
 0000:fffe0000       .debug$S                   00400000     vcruntime:VCRUNTIME140.dll
 0000:fffe0000       .debug$S                   00400000     vcruntime:VCRUNTIME140.dll
 0000:fffe0000       .debug$S                   00400000     vcruntime:VCRUNTIME140.dll
 0000:fffe0000       .debug$S                   00400000     ucrt:api-ms-win-crt-filesystem-l1-1-0.dll
 0000:fffe0000       .debug$S                   00400000     ucrt:api-ms-win-crt-string-l1-1-0.dll
 0000:fffe0000       .debug$S                   00400000     ucrt:api-ms-win-crt-stdio-l1-1-0.dll
 0000:fffe0000       .debug$S                   00400000     ucrt:api-ms-win-crt-runtime-l1-1-0.dll
 0000:fffe0000       .debug$S                   00400000     ucrt:api-ms-win-crt-runtime-l1-1-0.dll
 0000:fffe0000       .debug$S                   00400000     ucrt:api-ms-win-crt-runtime-l1-1-0.dll
 0000:fffe0000       .debug$S                   00400000     ucrt:api-ms-win-crt-runtime-l1-1-0.dll
 0000:fffe0000       .debug$S                   00400000     ucrt:api-ms-win-crt-runtime-l1-1-0.dll
 0000:fffe0000       .debug$S                   00400000     ucrt:api-ms-win-crt-runtime-l1-1-0.dll
 0000:fffe0000       .debug$S                   00400000     ucrt:api-ms-win-crt-runtime-l1-1-0.dll
 0000:fffe0000       .debug$S                   00400000     ucrt:api-ms-win-crt-runtime-l1-1-0.dll
 0000:fffe0000       .debug$S                   00400000     ucrt:api-ms-win-crt-stdio-l1-1-0.dll
 0000:fffe0000       .debug$S                   00400000     ucrt:api-ms-win-crt-heap-l1-1-0.dll
 0000:fffe0000       .debug$S                   00400000     ucrt:api-ms-win-crt-locale-l1-1-0.dll
 0000:fffe0000       .debug$S                   00400000     ucrt:api-ms-win-crt-runtime-l1-1-0.dll
 0000:fffe0000       .debug$S                   00400000     ucrt:api-ms-win-crt-runtime-l1-1-0.dll
 0000:fffe0000       .debug$S                   00400000     ucrt:api-ms-win-crt-runtime-l1-1-0.dll
 0000:fffe0000       .debug$S                   00400000     ucrt:api-ms-win-crt-runtime-l1-1-0.dll
 0000:fffe0000       .debug$S                   00400000     ucrt:api-ms-win-crt-runtime-l1-1-0.dll
 0000:fffe0000       .debug$S                   00400000     ucrt:api-ms-win-crt-stdio-l1-1-0.dll
 0000:fffe0000       .debug$S                   00400000     ucrt:api-ms-win-crt-runtime-l1-1-0.dll
 0000:fffe0000       .debug$S                   00400000     ucrt:api-ms-win-crt-runtime-l1-1-0.dll
 0000:fffe0000       .debug$S                   00400000     ucrt:api-ms-win-crt-runtime-l1-1-0.dll
 0000:fffe0000       .debug$S                   00400000     ucrt:api-ms-win-crt-runtime-l1-1-0.dll
 0000:fffe0000       .debug$S                   00400000     ucrt:api-ms-win-crt-runtime-l1-1-0.dll
 0000:fffe0000       .debug$S                   00400000     ucrt:api-ms-win-crt-runtime-l1-1-0.dll
 0000:fffe0000       .debug$S                   00400000     ucrt:api-ms-win-crt-math-l1-1-0.dll
 0000:fffe0000       .debug$S                   00400000     ucrt:api-ms-win-crt-runtime-l1-1-0.dll
 0000:fffe0000       .debug$S                   00400000     ucrt:api-ms-win-crt-runtime-l1-1-0.dll
 0000:fffe0000       .debug$S                   00400000     ucrt:api-ms-win-crt-time-l1-1-0.dll
 0000:fffe0000       .debug$S                   00400000     ucrt:api-ms-win-crt-stdio-l1-1-0.dll
 0000:fffe0000       .debug$S                   00400000     ucrt:api-ms-win-crt-stdio-l1-1-0.dll
 0000:fffe0000       .debug$S                   00400000     ucrt:api-ms-win-crt-string-l1-1-0.dll
 0000:fffe0000       .debug$S                   00400000     ucrt:api-ms-win-crt-runtime-l1-1-0.dll
 0000:fffe0000       .debug$S                   00400000     ucrt:api-ms-win-crt-heap-l1-1-0.dll
 0000:fffe0000       .debug$S                   00400000     ucrt:api-ms-win-crt-time-l1-1-0.dll
 0000:fffe0000       .debug$S                   00400000     ucrt:api-ms-win-crt-convert-l1-1-0.dll
 0000:fffe0000       .debug$S                   00400000     ucrt:api-ms-win-crt-utility-l1-1-0.dll
 0000:fffe0000       .debug$S                   00400000     ucrt:api-ms-win-crt-string-l1-1-0.dll
 0000:fffe0000       .debug$S                   00400000     ucrt:api-ms-win-crt-string-l1-1-0.dll
 0000:fffe0000       .debug$S                   00400000     ucrt:api-ms-win-crt-stdio-l1-1-0.dll
 0000:fffe0000       .debug$S                   00400000     ucrt:api-ms-win-crt-environment-l1-1-0.dll
 0000:fffe0000       .debug$S                   00400000     ucrt:api-ms-win-crt-runtime-l1-1-0.dll
 0000:fffe0000       .debug$S                   00400000     ucrt:api-ms-win-crt-string-l1-1-0.dll
 0000:fffe0000       .debug$S                   00400000     ucrt:api-ms-win-crt-string-l1-1-0.dll
 0000:fffe0000       .debug$S                   00400000     ucrt:api-ms-win-crt-string-l1-1-0.dll
 0000:fffe0000       .debug$S                   00400000     ucrt:api-ms-win-crt-string-l1-1-0.dll
 0000:fffe0000       .debug$S                   00400000     ucrt:api-ms-win-crt-runtime-l1-1-0.dll
 0000:fffe0000       .debug$S                   00400000     ucrt:api-ms-win-crt-stdio-l1-1-0.dll
 0000:fffe0000       .debug$S                   00400000     ucrt:api-ms-win-crt-stdio-l1-1-0.dll
 0000:fffe0000       .debug$S                   00400000     ucrt:api-ms-win-crt-filesystem-l1-1-0.dll
 0000:fffe0000       .debug$S                   00400000     ucrt:api-ms-win-crt-stdio-l1-1-0.dll
 0000:fffe0000       .debug$S                   00400000     ucrt:api-ms-win-crt-stdio-l1-1-0.dll
 0000:fffe0000       .debug$S                   00400000     ucrt:api-ms-win-crt-stdio-l1-1-0.dll
 0000:fffe0000       .debug$S                   00400000     ucrt:api-ms-win-crt-stdio-l1-1-0.dll
 0000:fffe0000       .debug$S                   00400000     ucrt:api-ms-win-crt-heap-l1-1-0.dll
 0000:fffe0000       .debug$S                   00400000     ucrt:api-ms-win-crt-heap-l1-1-0.dll
 0000:fffe0000       .debug$S                   00400000     ucrt:api-ms-win-crt-heap-l1-1-0.dll
 0000:fffe0000       .debug$S                   00400000     vcruntime:VCRUNTIME140.dll
 0000:fffe0000       .debug$S                   00400000     vcruntime:VCRUNTIME140.dll
 0000:fffe0000       .debug$S                   00400000     vcruntime:VCRUNTIME140.dll
 0001:00000000       _deflate_stored            00401000 f   deflate.obj
 0001:000003aa       _deflate_fast              004013aa f   deflate.obj
 0001:000006e6       _deflate_slow              004016e6 f   deflate.obj
 0001:000016d4       _deflateStateCheck         004026d4 f   deflate.obj
 0001:00001727       _deflate_huff              00402727 f   deflate.obj
 0001:0000188b       _deflate_rle               0040288b f   deflate.obj
 0001:00001b18       _fill_window               00402b18 f   deflate.obj
 0001:00001cbf       _flush_pending             00402cbf f   deflate.obj
 0001:00001d08       _lm_init                   00402d08 f   deflate.obj
 0001:00001d95       _longest_match             00402d95 f   deflate.obj
 0001:00001eff       _putShortMSB               00402eff f   deflate.obj
 0001:00001f29       _read_buf                  00402f29 f   deflate.obj
 0001:00001f93       _slide_hash                00402f93 f   deflate.obj
 0001:000039b4       $LN767                     004049b4     inflate.obj
 0001:00003c2a       _inflateStateCheck         00404c2a f   inflate.obj
 0001:00003c5d       _updatewindow              00404c5d f   inflate.obj
 0001:00004589       _bi_flush                  00405589 f   trees.obj
 0001:000045f5       _bi_windup                 004055f5 f   trees.obj
 0001:0000464c       _build_bl_tree             0040564c f   trees.obj
 0001:000046b2       _build_tree                004056b2 f   trees.obj
 0001:00004946       _compress_block            00405946 f   trees.obj
 0001:00004d0c       _detect_data_type          00405d0c f   trees.obj
 0001:00004d74       _gen_bitlen                00405d74 f   trees.obj
 0001:00004f90       _init_block                00405f90 f   trees.obj
 0001:00004fff       _pqdownheap                00405fff f   trees.obj
 0001:000050b6       _scan_tree                 004060b6 f   trees.obj
 0001:00005192       _send_all_trees            00406192 f   trees.obj
 0001:000053a5       _send_tree                 004063a5 f   trees.obj
 0001:00005d9c       _crc_word                  00406d9c f   zcrc32.obj
 0001:00006533       ?decode_sign@@YAHHI@Z      00407533 f   coding.obj
 0001:00006627       ?getDeltaValue@@YAHPAUvalue_stream@@I_N@Z 00407627 f   coding.obj
 0001:0000685b       $LN57                      0040785b     coding.obj
 0001:0000689b       ?getPopValue@@YAHPAUvalue_stream@@I@Z 0040789b f   coding.obj
 0001:00007474       ?init_args@@YAPAPADHPAPADAAH@Z 00408474 f   main.obj
 0001:00007596       ?nbasename@@YAPBDPBD@Z     00408596 f   main.obj
 0001:000075b0       ?next_arg@@YAHAAPAPAD@Z    004085b0 f   main.obj
 0001:000076b2       ?read_input_via_stdio@@YA_JPAUunpacker@@PAX_J2@Z 004086b2 f   main.obj
 0001:00007777       ?read_magic@@YAHPAUunpacker@@QADH@Z 00408777 f   main.obj
 0001:00007d3d       ?usage@@YAXPAUunpacker@@PBD_N@Z 00408d3d f   main.obj
 0001:00008177       ?compare_Utf8_chars@@YAHAAUbytes@@0@Z 00409177 f   unpack.obj
 0001:00009749       ?isDigitString@@YA_NAAUbytes@@HH@Z 0040a749 f   unpack.obj
 0001:000097a8       ?isLoadableValue@@YA_NH@Z  0040a7a8 f   unpack.obj
 0001:00009810       ?is_branch_op@@YA_NH@Z     0040a810 f   unpack.obj
 0001:00009830       ?is_local_slot_op@@YA_NH@Z 0040a830 f   unpack.obj
 0001:0000985a       ?lastIndexOf@@YAHHHAAUbytes@@H@Z 0040a85a f   unpack.obj
 0001:0000c403       $LN67                      0040d403     unpack.obj
 0001:0000d862       $LN21                      0040e862     unpack.obj
 0001:0000de6e       ?store_Utf8_char@@YAPACPACG@Z 0040ee6e f   unpack.obj
 0001:0000f42c       $LN53                      0041042c     unpack.obj
 0001:0000f448       $LN48                      00410448     unpack.obj
 0001:000105e0       ?read_input_via_gzip@@YA_JPAUunpacker@@PAX_J2@Z 004115e0 f   zip.obj
 0001:00010ea0       $$000000                   00411ea0     MSVCRT:llrem.obj
 0001:00010f60       $$000000                   00411f60     MSVCRT:llmul.obj
 0001:00010fa0       $$000000                   00411fa0     MSVCRT:ullshr.obj
 0001:00010fbf       ?pre_c_initialization@@YAHXZ 00411fbf f   MSVCRT:exe_main.obj
 0001:0001106a       ?post_pgo_initialization@@YAHXZ 0041206a f   MSVCRT:exe_main.obj
 0001:00011072       ?pre_cpp_initialization@@YAXXZ 00412072 f   MSVCRT:exe_main.obj
 0001:00011084       ?__scrt_common_main_seh@@YAHXZ 00412084 f   MSVCRT:exe_main.obj
 0001:00011210       ?find_pe_section@@YAPAU_IMAGE_SECTION_HEADER@@QAEI@Z 00412210 f   MSVCRT:utility.obj
 0001:0001148d       ___get_entropy             0041248d f   MSVCRT:gs_support.obj
 0001:000117b0       $$000000                   004127b0     MSVCRT:sehprolg4.obj
 0002:00000158       ?pre_cpp_initializer@@3P6AXXZA 00413158     MSVCRT:exe_main.obj
 0002:00000164       ?pre_c_initializer@@3P6AHXZA 00413164     MSVCRT:exe_main.obj
 0002:00000168       ?post_pgo_initializer@@3P6AHXZA 00413168     MSVCRT:exe_main.obj
 0002:000001d0       _configuration_table       004131d0     deflate.obj
 0002:00000248       ?my_version@?1??deflateInit2_@@9@9 00413248     deflate.obj
 0002:00000250       ?lenfix@?1??fixedtables@@9@9 00413250     infback.obj
 0002:00000a50       ?distfix@?1??fixedtables@@9@9 00413a50     infback.obj
 0002:00000ad0       ?order@?1??inflateBack@@9@9 00413ad0     infback.obj
 0002:00000c38       ?lenfix@?1??fixedtables@@9@9 00413c38     inflate.obj
 0002:00001438       ?distfix@?1??fixedtables@@9@9 00414438     inflate.obj
 0002:000014b8       ?order@?1??inflate@@9@9    004144b8     inflate.obj
 0002:000015b8       ?lbase@?1??inflate_table@@9@9 004145b8     inftrees.obj
 0002:000015f8       ?lext@?1??inflate_table@@9@9 004145f8     inftrees.obj
 0002:00001638       ?dbase@?1??inflate_table@@9@9 00414638     inftrees.obj
 0002:00001678       ?dext@?1??inflate_table@@9@9 00414678     inftrees.obj
 0002:000019b8       _extra_lbits               004149b8     trees.obj
 0002:00001a2c       _bl_order                  00414a2c     trees.obj
 0002:00001a40       _extra_dbits               00414a40     trees.obj
 0002:00001ab8       _extra_blbits              00414ab8     trees.obj
 0002:00001b08       _static_ltree              00414b08     trees.obj
 0002:00001f88       _static_dtree              00414f88     trees.obj
 0002:00002000       _base_length               00415000     trees.obj
 0002:00002078       _base_dist                 00415078     trees.obj
 0002:000020f0       _static_l_desc             004150f0     trees.obj
 0002:00002104       _static_d_desc             00415104     trees.obj
 0002:00002118       _static_bl_desc            00415118     trees.obj
 0002:00002130       _crc_table                 00415130     zcrc32.obj
 0002:00002530       _crc_big_table             00415530     zcrc32.obj
 0002:00002930       _crc_braid_table           00415930     zcrc32.obj
 0002:00003930       _crc_braid_big_table       00416930     zcrc32.obj
 0002:00004930       _x2n_table                 00417930     zcrc32.obj
 0002:00004a58       ?all_band_inits@@3QBUband_init@@B 00417a58     bands.obj
 0002:00006098       ?ERB@@3QBDB                00419098     coding.obj
 0002:000061a4       ?flag_opts@@3QBDB          004191a4     main.obj
 0002:000061ac       ?string_opts@@3QBDB        004191ac     main.obj
 0002:000061b0       ?sccsver@@3QBDB            004191b0     main.obj
 0002:00006748       ?TAGS_IN_ORDER@@3QBCB      00419748     unpack.obj
 0002:00006758       ?TAG_ORDER@@3QBCB          00419758     unpack.obj
 0002:0000676c       ?str_tf@@3QBDB             0041976c     unpack.obj
 0002:00007504       ?jarmagic@@3QBGB           0041a504     zip.obj
 0002:00007508       ?marker_comment@@3QBDB     0041a508     zip.obj
 0002:00007698       _GS_ExceptionPointers      0041a698     MSVCRT:gs_report.obj
 0002:00007a88       __sehtable$?__scrt_common_main_seh@@YAHXZ 0041aa88     MSVCRT:exe_main.obj
 0002:00007aa8       __sehtable$___scrt_is_nonwritable_in_current_image 0041aaa8     MSVCRT:utility.obj
 0002:00007ad0       .edata                     0041aad0     unpack200.exp
 0002:00007af8       rgpv                       0041aaf8     unpack200.exp
 0002:00007afc       rgszName                   0041aafc     unpack200.exp
 0002:00007b00       rgwOrd                     0041ab00     unpack200.exp
 0002:00007b02       szName                     0041ab02     unpack200.exp
 0002:00007b10       $N00001                    0041ab10     unpack200.exp
 0002:00007e9c       .idata$6                   0041ae9c     kernel32:KERNEL32.dll
 0002:00007ef6       .idata$6                   0041aef6     vcruntime:VCRUNTIME140.dll
 0002:00008208       .idata$6                   0041b208     ucrt:api-ms-win-crt-heap-l1-1-0.dll
 0002:00008228       .idata$6                   0041b228     ucrt:api-ms-win-crt-stdio-l1-1-0.dll
 0002:00008248       .idata$6                   0041b248     ucrt:api-ms-win-crt-filesystem-l1-1-0.dll
 0002:0000826e       .idata$6                   0041b26e     ucrt:api-ms-win-crt-runtime-l1-1-0.dll
 0002:00008290       .idata$6                   0041b290     ucrt:api-ms-win-crt-string-l1-1-0.dll
 0002:000082b2       .idata$6                   0041b2b2     ucrt:api-ms-win-crt-environment-l1-1-0.dll
 0002:000082d8       .idata$6                   0041b2d8     ucrt:api-ms-win-crt-utility-l1-1-0.dll
 0002:000082fa       .idata$6                   0041b2fa     ucrt:api-ms-win-crt-convert-l1-1-0.dll
 0002:0000831c       .idata$6                   0041b31c     ucrt:api-ms-win-crt-time-l1-1-0.dll
 0002:0000833c       .idata$6                   0041b33c     ucrt:api-ms-win-crt-math-l1-1-0.dll
 0002:0000835c       .idata$6                   0041b35c     ucrt:api-ms-win-crt-locale-l1-1-0.dll
 0003:00000af8       ?keys@?M@??next_arg@@YAHAAPAPAD@Z@4PAPBDA 0041caf8     main.obj
 0003:00000b18       ?opts@?1??dump_options@unpacker@@QAEXXZ@4PAPBDA 0041cb18     unpack.obj
 0003:00000b58       ?dummy@@3PACA              0041cb58     bytes.obj
 0003:00000f58       ?no_meta@@3PAPBCA          0041cf58     coding.obj
 0003:00000f60       ?suppress_warning@@3_NA    0041cf60     main.obj
 0003:00000f70       ?no_bands@@3PAPAUband@@A   0041cf70     unpack.obj
 0003:00000f78       _GS_ExceptionRecord        0041cf78     MSVCRT:gs_report.obj
 0003:00000fc8       _GS_ContextRecord          0041cfc8     MSVCRT:gs_report.obj
 0003:0000129c       ?is_initialized_as_dll@@3_NA 0041d29c     MSVCRT:utility.obj
 0003:0000129d       ?module_local_atexit_table_initialized@@3_NA 0041d29d     MSVCRT:utility.obj
 0003:000012a0       ?module_local_atexit_table@@3U_onexit_table_t@@A 0041d2a0     MSVCRT:utility.obj
 0003:000012ac       ?module_local_at_quick_exit_table@@3U_onexit_table_t@@A 0041d2ac     MSVCRT:utility.obj
 0004:00000060       $R000000                   0041e060     unpack200.exe.res
